:1062F600011900001D01010C0200000301FA04004F
:10630600FA0500030A0A5A0B001E0C00FA0D0003D8
:106316000E00040F0164100096120132130AFA14DB
:10632600010215000017010A1801FA1905321A01AF
:106336000A1B01FA1C05321FFFFF20FFFF23011E67
:106346002400642A00FA2B00FA2C50782D003D2EEA
:1063560000462F001E30006432507833000034327D
:10636600FA350164360164370150380A643C00642A
:106376003E003C3F000140FFFF411450420A5A4391
:106386000AC84405324500B44600FA4701184802D7
:10639600034C00FA4EFFFF500404510596520A3290
:1063A600530B46540A9656010257054658000259A1
:1063B6000A465A32FA5B010A5C0A325E000A5F003C
:1063C600FE61FFFF64010666000267FFFF6A0A3C82
:1063D6006B00006C3296730000740000780132790D
:1063E60001327EFFFF81FFFF84FFFF8500AF86003D
:1063F600018700FA89010A8A00009900009D0A9621
:106406009E00019FFFFFA0FFFFFAFAFA00001D01A0
:10641600010C0200000301FA0400FA0500030A0A4F
:106426005A0B001E0C00FA0D00030E00040F016447
:10643600100096120132130AFA1401021500001711
:10644600010A1801FA1905321A010A1B01FA1C057C
:10645600321FFFFF20FFFF23011E2400642A00FADB
:106466002B00FA2C50782D003D2E00462F001E30B2
:1064760000643250783300003432FA350164360154
:1064860064370150380A643C00643E003C3F00011A
:1064960040FFFF411450420A5A430AC84405324598
:1064A60000B44600FA4701184802024C00FA4EFFB3
:1064B600FF500404510596520A32530B46540A966D
:1064C600560101570546580001590A465A32FA5BE9
:1064D600010A5C0A325E000A5F00FE61FFFF64018A
:1064E6000666000267FFFF6A0A3C6B00006C329684
:1064F6007300007400007801327901327EFFFF815B
:10650600FFFF84FFFF85FFFF86FFFF87FFFF8901EF
:10651600028A00009900009D0A969E00019FFFFFD7
:10652600A0FFFFFAFAFA0065006F00790083008D7C
:10653600009700A100AC00B600C000CA00D400DE7F
:1065460000E800F2005800600068007000780080E3
:1065560000880090009800A000A800B000B800C114
:1065660000C800D000D800DF00E600EE00F60041CB
:106576000047004D00530059005F0065006C007134
:106586000077007D00830089008F0095009B00A2A4
:1065960000A700AC00B200B900C000C500CA00D216
:0A65A60000D500DD00E100E700EF82
:103A3900900049E0D3940440149007BAE0FEA3E053
:103A4900FF9062F81266E9E493F59980129007BA3B
:103A5900E0FEA3E0FF9064121266E9E493F5999001
:103A690007BAE0FEA3E0FF9062F6E493FC740193C9
:103A7900FDEFB50507EEB50403754D009007BA12C1
:103A890066D02285F97385FA747E017F00E5741288
:103A990066C2E5732FFF50010E8E5A8F5B9000139B
:103AA900E0FCA3E0FDEF2DFDEE3CFC8C5C8D5D227E
:103AB90075A71085F97385FA747E017F00E5741284
:103AC90066C2E5732FFF50010E8E5A8F5B9000DCA2
:103AD900E0B40210AC2CAD2DEF2DFDEE3CFC8C5C5E
:103AE9008D5D8016AE5AAF5B900013E0FCA3E0FD3C
:103AF900EF2DFDEE3CFC8C5C8D5D22AE5AAF5B7404
:103B09001E8E048F05FF1266B28C5C8D5DAE5AAFB6
:103B19005B741E8E048F05FF1266DD8C5A8D5BE582
:103B29005B455A6013741EC3955BFFE4955AFE8E7C
:103B39005A8F5B785C126716E573A85CB80015D3D9
:103B4900955D4010E573C3955DFFE4955CFE8E5C61
:103B59008F5D8010E573240CC3955DFFE4955CFED1
:103B69008E5C8F5D757300A21E4028AE5CAF5D74DC
:103B79000B6F4E6006740C6F4E7018AE5CAF5D74BF
:103B89000B6F4E70057573018003757302755D0ABD
:103B9900755C002290008AE0B40104C2108002D250
:103BA9001090008BE0B40104C2118002D211900080
:103BB900C8E075F0D2A4FFAEF0740A8E048F05FF39
:103BC9001266B29007B0ECF0A3EDF0A20D401674A6
:103BD900038C068D071266C274011200399007AE74
:103BE900EEF0A3EFF07E017F00900086E01266C23E
:103BF9009000C9E08E048F05FF1266B2740AFF12A5
:103C090066B28D609000D2E075F0D2A4FFAEF07478
:103C19000A8E048F05FF1266B29007B4ECF0A3ED8B
:103C2900F09000D4E060139000D4E0F5F0741684AD
:103C3900FF7E00EF9007C2F0800674649007C2F01F
:103C49009000CAE090006EF0900114E0900058F0E6
:103C59009000A3E090005AF09000CCE090005BF057
:103C6900900078E090005CF09000FEE0900061F038
:103C7900900162E0900062F0900163E0900063F0CF
:103C8900900164E0900064F0A227B34016900162AD
:103C9900E0700C900163E07006900164E0600280BE
:103CA90002C22774E390006DF09000B3E0B40B08F2
:103CB90074E390006DF0805A9000B3E0B41912904B
:103CC90000C9E090651712008CE49390006DF080B4
:103CD900419000B3E0B41E129000C9E0906535121E
:103CE900008CE49390006DF080289000B3E0B42834
:103CF900129000C9E090655F12008CE49390006D0A
:103D0900F0800F9000B3E0B446089000AAE090005C
:103D19006DF09000E3E0FE9000B1E06E600A900063
:103D2900B1E09000E3F0D226900071E0FE9000B07F
:103D3900E0B50633900073E0FE9000CEE0B50627AB
:103D4900900072E0FE9000DCE0B5061B900075E083
:103D5900FE900083E0B5060F900074E0FE9000BE6F
:103D6900E06E7003023EB0900049E0C3940550082C
:103D790074029000FFF080149000DCE06008740881
:103D89009000FFF08006740A9000FFF0900083E035
:103D9900B4010674009000E9F0900083E0B40206D3
:103DA90074009000CEF0900083E0B4030674009094
:103DB90000DBF09000CEE0D3940140147418900118
:103DC90001F074009006C8F074009006C9F0800CE8
:103DD9007400900101F074189006C8F09000B0E0EA
:103DE9006014741A900097F074009006D0F0740073
:103DF9009006D1F0800C7400900097F0741A900628
:103E0900D0F09000B0E0B402147419900098F074E6
:103E1900009006CCF074009006CDF0800C740090F0
:103E29000098F074199006CCF09000DCE0700E74E4
:103E3900059006DCF074069006E0F0801874009096
:103E490006DCF074009006DDF074009006E0F07472
:103E5900009006E1F0D2269000B0E0900071F09059
:103E690000DCE0900072F09000CEE0900073F090DA
:103E790000BEE0900074F0900083E0900075F0902F
:103E89000083E0900059F09000BEE090005DF09052
:103E990000DCE090005EF09000B0E090005FF090F0
:103EA90000CEE0900060F09000E6E0B401179000C9
:103EB9001F740FF0A374FFF0900021E4F0A3F074D5
:103EC900029000E6F09000E6E0B40341900021E0A2
:103ED900FEA3E0FF90001FE0FCA3E0FD12670E7453
:103EE900101266C27408120039EF90006AF0EF7080
:103EF9000674FF90006AF074009000E6F0900020CC
:103F0900E090006BF090001FE090006CF09000775B
:103F1900E090003BF090003BE0240690003CF090DC
:103F2900003CE0D3940C400B90003CE0C3940C900F
:103F3900003CF090003FE4F090003BE0640B600728
:103F490090003BE0B40C2090003BE0B40B067402F7
:103F590090003FF090003BE0B40C0690003F7401E4
:103F6900F090003B7401F0900040E4F090003CE0D8
:103F7900640B600790003CE0B40C2090003CE0B476
:103F89000B067402900040F090003CE0B40C0690DF
:103F990000407401F090003C7401F0900077E0FE5D
:103FA9009000DAE02E900042F0900042E064066052
:103FB90007900042E0B40C06900042E004F0900043
:103FC90042E064056007900042E0B40B06900042AD
:103FD900E014F0900042E0D3940C400B900042E0D2
:103FE900C3940C900042F0900042E0D39406400D37
:103FF900900042E0C39406900043F0800A9000428A
:10400900E02406900043F07551069000BDE0900051
:104019003DF090003DE075F00684AFF07E00EF4E74
:10402900700690003DE004F090003DE00475F00654
:1040390084AFF07E00EF4E700690003DE014F090E2
:10404900003DE0B4190690003D7401F090003DE098
:10405900D3940C400F90003DE0C3940C90003DF0C8
:10406900D2208002C22090003DE0D39406400D90FA
:10407900003DE0C3940690003EF0800A90003DE0C8
:10408900240690003EF022C293C294C291C292C209
:1040990087C290E5B554EFF5B5E5B554DFF5B5C27E
:1040A90096C295C2A0C297C2A2C2A1E5B554BFF5F6
:1040B900B5E5B5547FF5B5E5B554FBF5B5C212754F
:1040C9005E469000C0E07005756D028003756D0352
:1040D90075550075540090000874FFF0A374DCF066
:1040E900C217C21974C8900033F074C8900037F031
:1040F900755300755200C20D754600E56FB409038A
:10410900756F00756300900015E4F0A3F0757010E9
:10411900C215C2169007B0E0FEA3E0FF7403126651
:10412900C274011200399007AEEEF0A3EFF0C2029B
:1041390075570075560090000CE4F0A3F0C228757D
:104149005900755800900082E075F032A4FDACF07A
:1041590090001DECF0A3EDF0C238A22CB39205A299
:104169002DB39206A22EB39207A22FB39208A230C2
:10417900B39209A231B3920AA232B3920BA233B31A
:10418900920C2285F97385FA747E017F00E5741219
:1041990066C2E5732FFF50010E8E5A8F5BAC5CAD82
:1041A9005DEF2DFDEE3CFC8C5C8D5DD293D294E5E8
:1041B9005DF5FBE55CF5FCE55DF5E9E55CF5EA90A7
:1041C90000BEE0B40314D291D292E55DF5EBE55C53
:1041D900F5ECE55DF5EDE55CF5EE2275A71085F9E1
:1041E9007385FA747E017F00E5741266C2E5732F48
:1041F900FF50010E8E5A8F5B7E017F769000FBE0A7
:104209001266C2AC5AAD5BED2FFFEC3EFE8E5C8FA1
:104219005DE55DF5FDE55CF5FE90006EE4F075A7E2
:10422900007412900045F02285F97385FA747E01B5
:104239007F00E5741266C2E5732FFF50010E8E5A96
:104249008F5B9007B0E0FCA3E0FDEF2DFDEE3CFC99
:104259008C5C8D5DE55DF5FDE55CF5FE220564226E
:104269009000BEE0B403539000DCE0B4012EA2D864
:10427900B34004C293C287A2D9B34004C294C29086
:10428900A2DAB34008C291E5B554EFF5B5A2DBB3A4
:104299004008C292E5B554DFF5B5801CA2D8B340F9
:1042A90002C293A2D9B34002C294A2DAB34002C2B5
:1042B90091A2DBB34002C292801EA2D8B3400AC2C7
:1042C900939000DCE06002C287A2D9B3400AC2948D
:1042D9009000DCE06002C290A2DCB34004C296C246
:1042E9009575D8402285A77275A710A2D8B3400248
:1042F900C287A2D9B34002C290A2DAB34006E5B59B
:1043090054EFF5B5A2DBB34006E5B554DFF5B5A228
:10431900DCB340089000CAE090006EF075D8408583
:1043290072A722900047E4936406600280FE74C875
:104339009007B6F8E4F0E8A3F075B5007584017547
:10434900A70075FFA0900041E4F075C91075A70F8B
:1043590075A1C775A70075D90075CE0C75A70F751E
:10436900F1FE75F2FF75F30775F47875A4BA75A5B2
:10437900FF75A60775AE0075AFFF75D48175D5FFBA
:1043890075D6FF75D7FF75A70075A20175A1477589
:10439900F80975D80075D90475DA0975DB0975DC72
:1043A9000975DD0975DE0975D84075A71075D8003E
:1043B90075D90475DA0975DB0975DC0975DD0975C7
:1043C900DE0975D84075A70075E60875E71075BC54
:1043D9000175BE0475BD6C75BE0775BDA075BE08B7
:1043E90075BD0175BC0075BB1875BC2075BA08751B
:1043F900E88075D11375A70F75E10575E20075C7DA
:1044090040124090759700759780740A1266A275DC
:1044190097C0E5975420700280F8758F0275A70040
:10442900D2AF75980075A90C75A70F75AB4375AD1B
:10443900FB75AC1E75A71075C91875CA0075CB0038
:1044490075C80475A700758912758E04758C007579
:104459008A00C2A9D28C758D00758B00D2ABD28E21
:1044690075EF0675D944C29974C8F5097508001223
:1044790000E975B5001204E974639007B6F8E4F031
:10448900E8A3F012037574C89007B6F8E4F0E8A33E
:10449900F07464F5097508001200E9900059E0907C
:1044A9000083F0900083E0D39403400C74009000E3
:1044B90083F07400900059F0C21D900083E0905F72
:1044C9000AF82828738028A2B44002D21D802075DA
:1044D900A70F75F30F75A700A2A34002D21D800F85
:0F44E90075A70F75F31775A700A2A44002D21D87
:0C5F0A000244CE0244D00244D80244E914
:1044F800A21DB3405F757308E573D3940E5020E591
:10450800739007B6F8E4F0E8A3F01202447464F577
:10451800097508001200E97873740126F650D974F9
:10452800029000BFF0900059E0900083F090008363
:10453800E0905F16F8282873801674009000E9F060
:10454800800E74009000CEF0800674009000DBF0BE
:0C5F160002454002454202454A02455245
:10455800D21C805D757301E573D394075020E57311
:104568009007B6F8E4F0E8A3F01202447464F50981
:104578007508001200E97873740126F650D97401A1
:104588009000BFF0900059E0900083F0900083E025
:10459800905F22F8282873801674009000E9F08054
:0F45A8000E74009000CEF0800674009000DBF0DF
:0C5F220002459F0245A10245A90245B1BD
:1045B700C21C900058E0900114F0900059E0900060
:1045C70083F090005AE09000A3F090005BE0900029
:1045D700CCF090005CE0900078F090005DE09000F7
:1045E700BEF090005EE09000DCF090005FE090008D
:1045F700B0F0900060E09000CEF0900061E0900095
:10460700FEF0900062E0900162F0900063E090019C
:1046170063F0900064E0900164F0900162E0700C38
:10462700900163E07006900164E060028004C22795
:104637008002D2279000C9E07006740A9000C9F082
:104647009000AAE0700674E39000AAF09000B0E032
:1046570004900071F09000B1E09000E3F0123B9DF0
:10466700E5B54401F5B57406900047F07401900074
:1046770048F0740390004AF0740590004BF07453AF
:1046870090004CF0740590004DF0900049E0B404A0
:1046970006740490004DF0740190004EF074009081
:1046A7000053F07400900056F074FF900057F074B8
:1046B7003290014DF0743490014EF0742D90014FFB
:1046C700F07432900150F07420900151F0743490DE
:1046D7000152F07443900153F07479900154F074CF
:1046E7006C900155F07420900156F0744490015776
:1046F700F07469900158F0747A900159F0747A90C7
:10470700015AF0747990015BF09000E5E090006A3F
:10471700F090009CE090006BF090009DE090006CA2
:10472700F0A2B6B3920EA2B3B3920FA2A4B3922390
:10473700A2B4B39224A2A3B39225900066E4F075C5
:104747006F00743A900776F074FD900777F0900049
:1047570067E4F09007B0E0FEA3E0FF74031266C2BF
:1047670074011200399007AEEEF0A3EFF0756E01F9
:10477700900045E4F0C222756300C213D214C2024E
:10478700757100C22AD203C22BD204C22CD205C231
:104797002DD206C22ED207C22FD208C230D209C2EA
:1047A70031D20AC232D20BC233D20CC21EC21FC2CE
:1047B70020C221C22612009E755F00756B007561CD
:1047C7000075653275660075670075680075690064
:1047D700756A00900015E4F0A3F0756C00D2B2D2B0
:1047E700A4D2B0D2B1D2A3D2A7D2A6D2A5D2B79023
:1047F7000082E0D394FA400674FA900082F07E01BA
:104807007F0090006CE01266C290006BE02FFF50B3
:10481700010E90001FEEF0A3EFF0EFD394FFEE949C
:104827000F400790001FE4F0A3F090006AE07006C5
:1048370074FF90006AF09000BFE0D39402400674C2
:10484700019000BFF09000C0E07005756D02800315
:10485700756D039000C1E0D3940140067400900089
:10486700C1F09000C7E0C3940A5006740A9000C7CD
:10487700F09000D1E0700674019000D1F09000D163
:10488700E0B4FF0674FE9000D1F09000D8E0D39416
:10489700FE400674FE9000D8F09000FEE0D394022C
:1048A700400674019000FEF0900114E0D39401409B
:1048B700067401900114F074019000DEF074019009
:1048C70000DFF074009000E6F07400900102F074CD
:1048D70000900106F074299006BCF0742A9006C077
:1048E700F074179006C4F0741B9006D4F0741C90F3
:1048F70006D8F0D29C9000B1E0D39404400674042B
:104907009000B1F0E570D3941040037570109006D5
:10491700BDE0D3940C400674009006BDF09006C12C
:10492700E0D3940C400674009006C1F09006C5E0F1
:10493700D3940C400674009006C5F09006C9E0D3E6
:10494700940C400674009006C9F09006CDE0D3940D
:104957000C400674009006CDF09006D1E0D3940C7D
:10496700400674009006D1F09006D5E0D3940C4031
:104977000674009006D5F09006D9E0D3940C400653
:1049870074009006D9F09006DDE0D3940C400674CD
:10499700009006DDF09006E1E0D3940C4006740029
:1049A7009006E1F0D2EC75CF01A298B34005C2980A
:1049B700120646E54D6006A299B3B340028005C2D0
:1049C70099120C57E54E64016005E54EB404028068
:1049D700D5C28E7E107F00E5641266C2E58D75F044
:1049E70010A4FDACF0EF2DFDEE3CFCE58B75F0104F
:1049F70084FF7E00ED2FFFEC3EFE8E548F55D28E46
:104A07009000A3E060099000A3E0C3943D400280BA
:104A17005C9000171266D0900017E0FEA3E0FF90AD
:104A27000019E0FCA3E0FDEFB50542EEB5043EB288
:104A37001BA20DB3401975E700A21BB34008E5B5EB
:104A47004404F5B58006E5B554FBF5B575E7109058
:104A57000019E0FEA3E0FF90001BE0FCA3E0FDEFE0
:104A67002DFDEE3CFC900019ECF0A3EDF09000B0AA
:104A7700E060099000B0E0C394034002806F122DFC
:104A870096A20DB35009900066E0C39410400280CF
:104A97000690009AE0F545E54575F005A4FFAEF0F0
:104AA7009007B8EEF0A3EFF0900087E0C395614060
:104AB70007E55FC3956050079007B8E4F0A3F0AE31
:104AC7002EAF2F9007B8E0FCA3E0FDEFD39DEE9C3F
:104AD7004004C2A1800B900066E0C394195002D233
:104AE700A19000B0E0B40205A2A1B392A29000B0D9
:104AF700E0B4031C122EB1AE2EAF2F9007B8E0FC26
:104B0700A3E0FDEFD39DEE9C4004D2A18002C2A199
:104B1700A2B6300E01B3500302517BA2B6300E018C
:104B2700B3500302517BA2B6301001B35003024FBA
:104B37009F756E009000A3E0B43D1975E700A210C1
:104B4700B34008E5B554FBF5B58006E5B54404F573
:104B5700B575E710055EA212B3B35013AE54AF5547
:104B6700900008E0FCA3E0FDEDC39FEC9E4003022C
:104B77004C95E56DB4032EA228B34022E55EB40B35
:104B870003756D01E55EC3940B50069000457401F3
:104B9700F0E55ED3940B40067402900045F0755E15
:104BA70001D228805AE56DB40206756D01755E0B5A
:104BB700E55EB40B05755E018045900045E07030F9
:104BC700E55EC3940B50069000457401F0E55ED393
:104BD700940B40067402900045F0E55EC3940B50B9
:104BE70002D222E55ED3940B4002D222C296C2952E
:104BF7009000C0E0B401051240908003755E01AEDD
:104C070056AF57AC54AD55EF2DFDEE3CFC74028CFE
:104C1700068D071200398E568F579000A3E0600962
:104C27009000A3E0C3943D40028043900017E0FE4C
:104C3700A3E0FF9000A3E08E048F05FF1266B27415
:104C4700018C068D0712003990001BEEF0A3EFF0E0
:104C570090001BE0F8A3E0900019C8F0A3C8F090FB
:104C67000017E4F0A3F0C21BE5B554FBF5B5A2B4F9
:104C7700B34002C224A2A4B34002C223A2A3B340FA
:104C870002C225A222B34002C222D21E803AAE56E9
:104C9700AF57AC54AD55EF2DFDEE3CFC74018C06BF
:104CA7008D071200398E568F57E56DC39402500D4C
:104CB700AC54AD557498C39D743A9C400280091258
:104CC70040907406900045F0E55EB41712740390A7
:104CD7000045F0D2229000C0E0B40103124090E5F5
:104CE7005EB40D0FA21E40067405900045F0C21E6B
:104CF700755E01AE58AF59AC54AD55EF2DFDEE3C86
:104D0700FC8C588D59AE54AF55EFD39DEE9C401196
:104D170090000FE0FAA3E0FBEBC394E8EA940340AA
:104D270002800690000F1266D090000CE0FEA3E010
:104D3700FFAC54AD55EF2DFDEE3CFC90000CECF0B4
:104D4700A3EDF09000C0E0B40118AE54AF55740560
:104D57001266C27401120039900008EEF0A3EFF05A
:104D67008011AE54AF5574021266C2900008EEF07F
:104D7700A3EFF0C28E758D00758B007564007555B5
:104D870001755400D28EE55E240275F00384AFF0FE
:104D97007E00EF4E707590000CE0F8A3E090000ADB
:104DA700C8F0A3C8F090000AE0FEA3E0FFEF4E6052
:104DB7000B7C7E7D801265B08E528F5390000CE481
:104DC700F0A3F0AE52AF537428BE00039F5010E516
:104DD700632FFF50010E74011200398E528F5385D5
:104DE70053639000C7E0A852B8000DD3955340080D
:104DF700E553900044F080099000C7E01490004408
:104E0700F0E56D60067553007552009000BEE0B482
:104E1700030890003DE0655E6002800BA21FB3406F
:104E270004D2218002B221E55E64046005E55EB428
:104E37000A099000B0E060031223D2900042E065B7
:104E47005E6007900043E0B55E03756F00A213B381
:104E57005006A212B3B34003024F0790007CE0B4A0
:104E670001739000FEE0B40214120E2690006FE06A
:104E770075F0BEA4FFAEF08E5C8F5D8056E567755A
:104E8700F00A84FF7E009005761266E9E0F55B750F
:104E97005A00AE5AAF5B9000A1E01266C274648EEE
:104EA700048F05FF1266B28C5C8D5DE55D90000E88
:104EB700F0AE5AAF5B90007AE01266C274648E045B
:104EC7008F05FF1266B274BE8C068D071266C28EFE
:104ED7005C8F5D801790007AE075F0BEA4FFAEF09E
:104EE7008E5C8F5D9000A1E090000EF0E561C394A9
:104EF700CC5006E55D455C7002800312418CD213ED
:104F0700E56DB40106E55E64046002800975700111
:104F17009000467401F0E56D70799000C3E0600D74
:104F270090006EE0A852B800069553400280389072
:104F370000C3E0B4021790003BE0655E6007900095
:104F47003CE0B55E03757003756C00800CC200759C
:104F57006C00900015E4F0A3F090006EE06006741A
:104F670009900045F0802C90003BE0655E6007905B
:104F7700003CE0B55E0375700190003BE0B55E064E
:104F87009000467401F090003CE0B55E0674029014
:104F97000046F0A210B3920EA210B330B601B35080
:104FA7000302517B756E019000A3E0B43D1975E7CC
:104FB70000A210B34008E5B54404F5B58006E5B591
:104FC70054FBF5B575E710E5B54401F5B5741090D8
:104FD7000066F0A210920EE55ED394484014D212F8
:104FE700E55ED3945F400B7405900045F0D22275BF
:104FF7005E469000CBE0B40107E56AC39414400213
:1050070080091240907413900045F0A22A300301E2
:10501700B3501D75E700A22AB34008E5B54408F56B
:10502700B58006E5B554F7F5B575E710A22A9203E2
:10503700A22B300401B3501D75E700A22BB3400823
:10504700E5B54402F5B58006E5B554FDF5B575E758
:1050570010A22B9204A22C300501B3500FA22CB33F
:105067004004D2A08002C2A0A22C9205A22D300635
:1050770001B3500FA22DB34004D2978002C297A26A
:105087002D9206A22E300701B3500FA22EB3400473
:10509700D2A28002C2A2A22E9207A22F300801B389
:1050A700500FA22FB34004D2A18002C2A1A22F9217
:1050B70008A230300901B3501D75E700A230B34094
:1050C70008E5B54440F5B58006E5B554BFF5B575B7
:1050D700E710A2309209A231300A01B3501D75E7DB
:1050E70000A231B34008E5B54480F5B58006E5B5C3
:1050F700547FF5B575E710A231920AA232300B0141
:10510700B3500FA232B34004D2878002C287A232C3
:10511700920BA233300C01B3500FA233B34004D229
:10512700908002C290A233920CE56AC39441500961
:10513700740E900045F012409090004DE0FE9000F4
:1051470049E004C39E4009900049E0D39408400910
:1051570074FB900045F0124090900052E06015906B
:105167000052E0FE90004CE06E600974FE9000452E
:10517700F0124090A222B34004C296C2959000FB61
:10518700E0600CAE52AF537414BE00059F4002801E
:1051970048900083E0905F2EF8282873803BA2B4E4
:1051A700B35005A224B3400280051241E4D2248003
:1051B70028A2A3B35005A225B3400280051241E4FB
:1051C700D2258015A2A4B35005A223B340028005BF
:0951D7001241E4D22380028000A1
:105F2E000251A30251A50251B80251CB0251DE0219
:025F3E0051E030
:1051E000A215B3B3500890003DE0655E6003025223
:1051F000BFA201B35006A200B3B340030252BB905A
:1052000000BEE0B403028003025290A20DB34067D7
:10521000A221B3402D123A8CE55DF5FBE55CF5FC6F
:10522000D293A202B34002D2879000DCE0B4021015
:10523000123AB9E55DF5FBE55CF5FC75A700D28790
:105240008033123A8CE55DF5EBE55CF5ECD291A28A
:1052500002B34006E5B54410F5B59000DCE0B402B9
:1052600014123AB9E55DF5EBE55CF5EC75A700E5E0
:10527000B54410F5B58017123A8CE55DF5FBE55C99
:10528000F5FCE55DF5EBE55CF5ECD293D291802B76
:10529000123A8CE55DF5FBE55CF5FCD293A202B316
:1052A0004002D2879000DCE0B40210123AB9E55D0A
:1052B000F5FBE55CF5FC75A700D287C215D216A2F6
:1052C00016B3B3500890003EE0655E600302539E43
:1052D000A201B35006A200B3B3400302539A900058
:1052E000BEE0B40302800302536FA20DB34067A275
:1052F00021B3402D123A8CE55DF5E9E55CF5EAD283
:1053000094A202B34002D2909000DCE0B4021012EA
:105310003AB9E55DF5E9E55CF5EA75A700D290805C
:1053200033123A8CE55DF5EDE55CF5EED292A20222
:10533000B34006E5B54420F5B59000DCE0B40214B6
:10534000123AB9E55DF5EDE55CF5EE75A700E5B55A
:105350004420F5B58017123A8CE55DF5E9E55CF57A
:10536000EAE55DF5EDE55CF5EED294D292802B1284
:105370003A8CE55DF5E9E55CF5EAD294A202B3402A
:1053800002D2909000DCE0B40210123AB9E55DF56B
:10539000E9E55CF5EA75A700D290D215C216E57072
:0E53A000905F40F828287302581B9000B1E07F
:065F40000253A70253AA60
:1053AE00905F73F8282873121EAE8012121EAE8004
:0E53BE000D121F388008121FE48003121FE436
:0F5F73000253B50253BA0253BF0253C40253C9BB
:1053CC0075700202581B122110122227A238B3400A
:1053DC00229000A5E0F56C900076E0256CFE900024
:1053EC0044E075F01E84FC7F00EE2CF536741090B2
:1053FC000045F09007AEE0FEA3E0FF740A1266C20F
:10540C0090000AE0FCA3E0FD74098F02FF1266B263
:10541C008D078C038E048A058B061265B09007B23B
:10542C00EEF0A3EFF09000CCE0B401087478BE006D
:10543C00059F4002800D74789007B2F8E4F0E8A361
:10544C00F0801B9007B2E0FEA3E0FF74F0BE0003F7
:10545C009F500B74F09007B2F8E4F0E8A3F0E53637
:10546C0070037536019007B2E0FEA3E0FFE5362F1E
:10547C00FF50010E9007B2EEF0A3EFF075700390A1
:03548C000046E0F7
:035F46000253D231
:10548F00905F82F82828738010A239400375700A44
:09549F008007A239400375700B6F
:095F82000254960254980254A145
:1054A80002581B9006BDE060031224EA9000FCE05D
:1054B800B401149000FDE0A852B8000495535007B9
:1054C800E55FC39560400280097415900045F002BD
:1054D800555B9000B1E0D39402403F900085E024F2
:1054E80003A852B8000495535009900087E0D3955B
:1054F8006150028008D2017408900045F090008540
:10550800E0A852B80005D39553500B900087E024CB
:1055180003C395615002C2018039900085E02403DD
:10552800A852B8000495535007E55FC39560400240
:105538008008D2017408900045F0900085E0A852D8
:10554800B80005D395535009E560240FC3955F5003
:1055580002C2019000CBE07007E56AC394144002D0
:105568008002D201A2014005757004800A7570108E
:10557800900015E4F0A3F0A20DB34029E56775F09B
:105588000A84FF7E009005761266E9E0C3946950AC
:1055980005122407800F9007B0E0F8A3E09007AE4B
:0C55A800C8F0A3C8F002581B9000B1E04E
:065F49000254AB0255B04A
:1055B400905F8BF8282873120F108012120F10803E
:0E55C4000D1210BE80081211708003121170BB
:0F5F8B000255BB0255C00255C50255CA0255CF7B
:1055D2009006C1E060031225C675700502581B12C1
:1055E20012B07570069006C5E060031226B69006EA
:1055F200C9E0600312279202581B90000EE0600679
:10560200A20DB3B34002801D90000EE02529FFAE2B
:105612002850010E8E288F29E55ED39406500690FD
:10562200000EE014F01214F67570079006CDE060DB
:105632000312286E9006D1E0600312294A02581B19
:105642009000FEE0B40203120E9E1218F575700867
:105652009006D5E06003122A269006D9E060031274
:105662002B0202581B121CB1A215B35005A216B38D
:1056720040028004D215D2167570109006DDE060EB
:1056820003122BDE9006E1E06003122CBA02581BD3
:1056920002581B900035E0C394465008C2967446E7
:1056A200900035F090003FE0B4011DE536241EF570
:1056B200369007B2E0FEA3E0FF741E2FFF50010EEA
:1056C2009007B2EEF0A3EFF090003FE0B4021DE5C8
:1056D20036243CF5369007B2E0FEA3E0FF743C2F7F
:1056E200FF50010E9007B2EEF0A3EFF085365B7526
:1056F2005A0090003BE0F573123B04E55D900035E3
:10570200F0900004E55AF0A3E55BF0E573900036F3
:10571200F0C2189007B2E0F55AA3E0F55B90003BA7
:10572200E0F573123B04E55D900033F0900000E574
:105732005AF0A3E55BF0E573900034F0C217E56D13
:10574200B4010575700B800375700302581B90003D
:1057520039E0C3944650139000CCE0B40104C296E1
:105762008002C2957446900039F0900040E0B40186
:105772001DE536241EF5369007B2E0FEA3E0FF7465
:105782001E2FFF50010E9007B2EEF0A3EFF0900033
:1057920040E0B4021DE536243CF5369007B2E0FE47
:1057A200A3E0FF743C2FFF50010E9007B2EEF0A36E
:1057B200EFF085365B755A0090003CE0F573123BC2
:1057C20004E55D900039F0900006E55AF0A3E55B30
:1057D200F0E57390003AF0C21A9007B2E0F55AA3CE
:1057E200E0F55B90003CE0F573123B04E55D900050
:1057F20037F0900002E55AF0A3E55BF0E573900004
:1058020038F0C219E56DB40103756D00757003803F
:0958120008800680048002800079
:105F4F000255E10255FC0256420256670256920272
:105F5F0056950257500258130258150258170258F7
:045F6F001902581BA0
:10581B00900033E0B55E0280030258CAA217407FA6
:10582B00900000E0FEA3E0FFEF4E602EAC56AD57AC
:10583B007405FF1266B28D068C07900000E0FCA386
:10584B00E0FDCFCECF12000374068E048F05FF123E
:10585B0066B2900000ECF0A3EDF0900034E0601A1B
:10586B00900000E0FEA3E0FFAC56AD57EF2DFDEE30
:10587B003CFC900000ECF0A3EDF0900034E0D394EE
:10588B0001401A900000E0FEA3E0FFAC56AD57EFCD
:10589B002DFDEE3CFC900000ECF0A3EDF0D217AE2A
:1058AB0054AF55900000E0FCA3E0FDEFC39DEE9CD0
:1058BB00400D124231D296C21774C8900033F0A239
:1058CB0017B3B35007900033E0B55E02800D124260
:1058DB0031D29674C8900033F0C217900035E0B502
:1058EB005E028003025992A218407F900004E0FEF2
:1058FB00A3E0FFEF4E602EAC56AD577405FF12665A
:10590B00B28D068C07900004E0FCA3E0FDCFCECF58
:10591B0012000374068E048F05FF1266B29000040A
:10592B00ECF0A3EDF0900036E0601A900004E0FE7E
:10593B00A3E0FFAC56AD57EF2DFDEE3CFC90000401
:10594B00ECF0A3EDF0900036E0D39401401A9000F8
:10595B0004E0FEA3E0FFAC56AD57EF2DFDEE3CFC93
:10596B00900004ECF0A3EDF0D218AE54AF559000BC
:10597B0004E0FCA3E0FDEFC39DEE9C400AC29674CD
:10598B0046900035F0C218A218B3B35007900035FB
:10599B00E0B55E02800AC2967446900035F0C218DC
:1059AB00900037E0B55E028003025A65A219407F72
:1059BB00900002E0FEA3E0FFEF4E602EAC56AD5719
:1059CB007405FF1266B28D068C07900002E0FCA3F3
:1059DB00E0FDCFCECF12000374068E048F05FF12AD
:1059EB0066B2900002ECF0A3EDF0900038E0601A84
:1059FB00900002E0FEA3E0FFAC56AD57EF2DFDEE9D
:105A0B003CFC900002ECF0A3EDF0900038E0D39456
:105A1B0001401A900002E0FEA3E0FFAC56AD57EF39
:105A2B002DFDEE3CFC900002ECF0A3EDF0D219AE94
:105A3B0054AF55900002E0FCA3E0FDEFC39DEE9C3C
:105A4B0040181242319000CCE0B40104D29680028F
:105A5B00D295C21974C8900037F0A219B3B350078E
:105A6B00900037E0B55E0280181242319000CCE016
:105A7B00B40104D2968002D29574C8900037F0C25C
:105A8B0019900039E0B55E028003025B43A21A4015
:105A9B007F900006E0FEA3E0FFEF4E602EAC56AD0C
:105AAB00577405FF1266B28D068C07900006E0FC5A
:105ABB00A3E0FDCFCECF12000374068E048F05FF3B
:105ACB001266B2900006ECF0A3EDF090003AE060A5
:105ADB001A900006E0FEA3E0FFAC56AD57EF2DFD8C
:105AEB00EE3CFC900006ECF0A3EDF090003AE0D316
:105AFB009401401A900006E0FEA3E0FFAC56AD57B0
:105B0B00EF2DFDEE3CFC900006ECF0A3EDF0D21A6D
:105B1B00AE54AF55900006E0FCA3E0FDEFC39DEE45
:105B2B009C40159000CCE0B40104C2968002C29553
:105B3B007446900039F0C21AA21AB3B35007900002
:105B4B0039E0B55E0280159000CCE0B40104C2963A
:105B5B008002C2957446900039F0C21A9000CEE0D4
:105B6B00B402028003025C83900068E0D395665018
:105B7B0064900068E0F4042566FE9000D1E08E008E
:105B8B00F5F0E884FF7E008F73EFC39410500CEF99
:105B9B008573F0A4FDACF08D7380037573FF9000DB
:105BAB0068E0D39573400B900068E0C39573F57173
:105BBB0080037571009000ECE0D395714006900066
:105BCB00ECE0F5719000EDE0C3957150069000ED9F
:105BDB00E0F5718071900068E0C39566FE9000D18E
:105BEB00E08E00F5F0E884FF7E008F73EFC3941016
:105BFB00500CEF8573F0A4FDACF08D7380037573BF
:105C0B00FF85735B755A00900068E0255BFFAE5A09
:105C1B0050010E8E5A8F5B74FFBE0009D39F400557
:105C2B00855B7180037571FF9000ECE0D39571403B
:105C3B00069000ECE0F5719000EDE0C39571500615
:105C4B009000EDE0F571A20DB3B3500D900069E03B
:105C5B00FE9000D9E0D39E5002800A740790004555
:105C6B00F0C297801375A710E5CDC395714004C2A0
:105C7B00978002D29775A700E56FC39409500AA2CB
:105C8B00EDB34005C2ED123050AE54AF5574C8C3DE
:105C9B009F74AF9E400C900067E0C3945A40030280
:105CAB005F07A212B340091240907406900045F0B2
:105CBB00A21DB34008E5B54404F5B58006E5B5541F
:105CCB00FBF5B5A214B3500EE561D394334007E551
:105CDB0061C394CC400280419000FEE0B4021412E8
:105CEB000E2690006FE075F050A4FFAEF08E5C8F27
:105CFB005D800F90007AE075F050A4FFAEF08E5CE3
:105D0B008F5DE55D455C6011E5B54401F5B574103B
:105D1B00900066F012418CD214900067E0D394018E
:105D2B004007E561C3941A40028002C2149006BD7D
:105D3B00E060031224EAA22A300301B35017A22A0F
:105D4B00B34008E5B54408F5B58006E5B554F7F55D
:105D5B00B5A22A92039006C1E060031225C6A22BBE
:105D6B00300401B35017A22BB34008E5B54402F53C
:105D7B00B58006E5B554FDF5B5A22B92049006C58A
:105D8B00E060031226B6A22C300501B3500FA22CF3
:105D9B00B34004D2A08002C2A0A22C92059006C9E7
:105DAB00E06003122792A22D300601B3500FA22DF3
:105DBB00B34004D2978002C297A22D92069006CDD3
:105DCB00E0600312286EA22E300701B3500FA22EF3
:105DDB00B34004D2A28002C2A2A22E92079006D197
:105DEB00E0600312294AA22F300801B3500FA22FF3
:105DFB00B34004D2A18002C2A1A22F92089006D573
:105E0B00E06003122A26A230300901B35017A230EA
:105E1B00B34008E5B54440F5B58006E5B554BFF58C
:105E2B00B5A23092099006D9E06003122B02A23181
:105E3B00300A01B35017A231B34008E5B54480F5E1
:105E4B00B58006E5B5547FF5B5A231920A9006DD13
:105E5B00E06003122BDEA232300B01B3500FA232E3
:105E6B00B34004D2878002C287A232920B9006E124
:105E7B00E06003122CBAA233300C01B3500FA233E3
:105E8B00B34004D2908002C290A233920C90006770
:105E9B00E0C3945A5010E56FB40909900067E00411
:105EAB00F0756F00803BE56FB40903756F00755596
:105EBB0000755400758D00758B007564009000663D
:105ECB00E0C394195008900066E004F08006741942
:105EDB00900066F0900066E0B41906E5B554FEF547
:105EEB00B5900067E0D394014007E56AC394414045
:0F5EFB00028009740E900045F01240900249ADEC
:105F9A000000010001400160018001A001C001E090
:105FAA0002000300039603B603D603F404000500B7
:105FBA000512052405360548055A056C057E059027
:105FCA0005A805C005DE0600061406280646066E64
:105FDA0006AE05CF00FF013F015F017F019F01BFB0
:105FEA0001DF01FF02FF039503B503D503F303FFA6
:105FFA0004FF05110523053505470559056B057D80
:10600A00058F05A705BF05CE05F106130627064528
:10601A00066D06AD06ED05DD0FAA0FA50F9F0F9AB7
:10602A000F940F8D0F870F800F780F710F680F6015
:10603A000F570F4E0F450F3B0F300F250F1A0F0E3C
:10604A000F020EF50EE80EDB0ECC0EBE0EAE0E9F44
:10605A000E8E0E7D0E6C0E5A0E470E340E200E0C4E
:10606A000DF70DE20DCB0DB50D9D0D850D6D0D5482
:10607A000D3A0D200D050CE90CCE0CB10C940C76E2
:10608A000C580C3A0C1B0BFB0BDB0BBB0B9A0B795A
:10609A000B570B350B130AF10ACE0AAB0A870A64AF
:1060AA000A400A1C09F809D409B0098C096709438E
:1060BA00091F08FB08D608B2088E086A0846082392
:1060CA0007FF07DC07B9079607730751072F070D64
:1060DA0006EC06CA06AA068906690649062A060AB7
:1060EA0005EC05CD05B0059205750558053C05205A
:1060FA00050504EA04CF04B5049C0482046904512A
:10610A0004390422040B03F403DE03C803B2039D1B
:10611A00038903750361034D033B03280316030434
:10612A0002F202E102D102C002B002A0029102828E
:10613A000273026502570249023C022F022202162A
:10614A00020901FD01F201E601DB01D001C601BB32
:10615A0001B101A7019D0194018B018201790170AE
:10616A0001680160015801500148014101390132B9
:10617A00012B0125011E01180111010B010500FF68
:10618A0000FA0FA60FA00F990F920F8B0F840F7CA6
:10619A000F740F6B0F620F580F4E0F430F380F2CEF
:1061AA000F1F0F120F050EF70EE80ED80EC80EB706
:1061BA000EA50E930E800E6C0E580E420E2C0E1566
:1061CA000DFD0DE40DCB0DB10D950D790D5D0D3F56
:1061DA000D200D010CE10CC00C9E0C7C0C590C35E9
:1061EA000C100BEA0BC40B9E0B760B4F0B260AFD09
:1061FA000AD40AAA0A800A550A2A09FF09D409A850
:10620A00097C0950092508F908CD08A10875084A2A
:10621A00081E07F307C8079D07730749072006F7F3
:10622A0006CE06A6067E06570630060A05E405BF10
:10623A00059B057705540532051004EF04CE04AE1C
:10624A00048F047104530435041903FD03E203C7E0
:10625A0003AD0394037B0363034B0334031E030858
:10626A0002F302DE02CA02B602A30291027F026DA3
:10627A00025C024C023C022C021D020E020001F2D8
:10628A0001E401D701CA01BE01B101A6019A018F39
:10629A000185017A01700166015D0153014A0141DC
:1062AA00013901310129012101190112010B0104EE
:1062BA0000FD00F700F000EA00E400DE00D900D398
:1062CA0000CE00C900C400BF00BA00B500B100ADDD
:1062DA0000A800A400A0009C009900950091008EDF
:0C62EA00008A008700840081007E007B99
:10009E007547009007BAE4F0A3F075310075300093
:1000AE00754D00754E00C235D23674FE9007BCF801
:1000BE00E4F0E8A3F074FE9007BEF8E4F0E8A3F0D5
:1000CE0074FE9007C8F0745A9007C9F0745A9007DE
:1000DE00CAF0D237C229C239C23422750B00750A52
:1000EE0000AE0AAF0BAC08AD09EDC39FEC9E4016F7
:1000FE0074FF1266A275CF01780B740126F65004B8
:10010E0018E436F650DB22900041E0B4AA1C9007AA
:10011E0076E0B43C159007B6E0FEA3E0FFEF4E602C
:10012E0009741EBE0004D39F5003020243755D0086
:10013E00755C0075F8099007B6E0FEA3E0FF740742
:10014E006F4E6006740E6F4E7006743A900776F01E
:10015E009007B6E0FEA3E0FF7408BE001ED39F40DA
:10016E001A7E017F089007B6E0FCA3E0FD1DBDFFDF
:10017E00011C1200038E5A8F5B801F9007B6E0FEA3
:10018E00A3E0FF74081267068F048E057E017F08B8
:10019E00CDCCCD1200038E5A8F5BAE5CAF5D740C6E
:1001AE00D39F74019E500302023EA2F9B3407EE536
:1001BE005D455C700375A382AE5CAF5D74016F4EDE
:1001CE00700375A300AE5CAF5D74026F4E700D9040
:1001DE0007B7E075F002A4FDACF08DA3AE5CAF5D89
:1001EE0074036F4E700375A300AE5CAF5D7403BEF7
:1001FE0000039F5013AC5AAD5BED2FFFEC3EFE900B
:10020E0000721266E9E0F5A3AE5CAF5DEFB40B09C8
:10021E00EEB4010574141266A2AE5CAF5DEFB40BC2
:10022E0007EEB4010375F80D785C1267160201A88B
:10023E00900041E4F022755D00755C0075F8099040
:10024E0007B6E0FEA3E0FF7408BE001ED39F401A5F
:10025E007E017F089007B6E0FCA3E0FD1DBDFF0107
:10026E001C1200038E5A8F5B801F9007B6E0FEA310
:10027E00E0FF74081267068F048E057E017F08CD9D
:10028E00CCCD1200038E5A8F5BAE5CAF5D7411D372
:10029E009F74019E5003020374A2F9B3500302032C
:1002AE0071E55D455C700375A3D2AE5CAF5D740104
:1002BE006F4E700375A300AE5CAF5D74026F4E702F
:1002CE000D9007B7E075F002A4FDACF08DA3AE5C07
:1002DE00AF5D74036F4E700375A300AE5CAF5D74BB
:1002EE00046F4E700375A300AE5CAF5D74056F4E68
:1002FE00700375A300AE5CAF5D74066F4E70037530
:10030E00A300AE5CAF5D74076F4E700375A300AEB5
:10031E005CAF5D74086F4E700375A300AE5CAF5D8D
:10032E007408BE00039F5016AC5AAD5BED2FFFEC68
:10033E003EFE90006D1266E9E5A3F075A300AE5C7B
:10034E00AF5DEFB41009EEB4010574141266A2AEDF
:10035E005CAF5DEFB41007EEB4010375F80D785C79
:10036E0012671602029722755D00755C0075F8091A
:10037E00AE5CAF5D7417BE0004D39F500302044DF4
:10038E00A2F9B3500302044AE55D455C700375A300
:10039E00D2AE5CAF5D74016F4E700375A300AE5CA0
:1003AE00AF5D74026F4E700D9007B7E075F002A44A
:1003BE00FDACF08DA3AE5CAF5D74036F4E70037534
:1003CE00A300AE5CAF5D74046F4E700375A300AEF8
:1003DE005CAF5D74056F4E700375A300AE5CAF5DD0
:1003EE0074066F4E700375A300AE5CAF5D74076F3D
:1003FE004E700375A300AE5CAF5D74086F4E700354
:10040E0075A300AE5CAF5D7408BE00039F500C90E8
:10041E00004F1266E9E5A3F075A300AE5CAF5D7404
:10042E00166F4E700574141266A2AE5CAF5D741634
:10043E006F4E700375F80D785C12671602037E22FC
:10044E00900041E0B4AB0280030204E8755D0075D4
:10045E005C0075F809AE5CAF5D7412BE007CD39F74
:10046E004078A2F9B34070E55D455C700375A382D8
:10047E00AE5CAF5D74016F4E700375A300AE5CAFE2
:10048E005D74026F4E700D9007B7E075F002A4FD1B
:10049E00ACF08DA3AE5CAF5D74036F4E700375A3AD
:1004AE0000AE5CAF5D7403BE00039F500990005414
:1004BE001266E9E0F5A3AE5CAF5D74116F4E700588
:1004CE0074141266A2AE5CAF5D74116F4E7003753C
:1004DE00F80D785C126716020463229007C5E4F0EB
:1004EE0074649007B6F8E4F0E8A3F012037574C8CC
:1004FE009007B6F8E4F0E8A3F074FF90004FF074A4
:10050E00FF900050F074FF900051F074009000497D
:10051E00F074FF900052F07400900054F07401904B
:10052E000055F090005BE0B4371A900058E0900050
:10053E004FF0900059E0900050F090005AE090007B
:10054E0051F080469007C57401F074659007B6F8B7
:10055E00E4F0E8A3F012037574C89007B6F8E4F05F
:10056E00E8A3F090005BE0B4371A900058E09000DA
:10057E004FF0900059E0900050F090005AE090003B
:10058E0051F0800674029007C5F09007C6E4F0742F
:10059E00669007B6F8E4F0E8A3F012037574C890FD
:1005AE0007B6F8E4F0E8A3F090005AE0B4371290E2
:1005BE000058E0900049F0900059E0900052F08011
:1005CE00769007C67401F074679007B6F8E4F0E809
:1005DE00A3F012037574C89007B6F8E4F0E8A3F020
:1005EE0090005AE0B43712900058E0900049F09015
:1005FE000059E0900052F0803E74029007C6F074ED
:10060E00689007B6F8E4F0E8A3F012037574C8908A
:10061E0007B6F8E4F0E8A3F090005AE0B437129071
:10062E000058E0900049F0900059E0900052F080A0
:10063E000674039007C6F022E54E64046006E59941
:10064E0064FF60028031A2354004D2358027E54E2A
:10065E00600874E6254E900045F0E54D600874F094
:10066E00254D900045F0E54EB4010280FE754E001A
:10067E00754D00C2358002C235E54E90384AF828D5
:10068E002873754E00E599B4FF03754D01E599B4D5
:10069E00FE03754D02E599B4FD03754D03E599B45E
:1006AE00FC03754D04E599B4FA03754D05E599B44F
:1006BE00FB06754E01124090E599B4F906754E048D
:1006CE00124090E599D394E54007E599C394F04024
:1006DE0002801685994F754E027E017F00E54FC34D
:1006EE0094E61266C28E328F339007BAE4F0A3F00E
:1006FE00E599D394C44007E599C394E64002802857
:10070E0085994F754E0374E5C3954FF533753200D9
:10071E00AE32AF33905F9A126691E493F874019300
:10072E009007BAC8F0A3C8F0D299020C56900058A0
:10073E00E07005A227B3400280429007BAE0FEA304
:10074E00E0FF74FFBE00039F5009EFC39446EE9482
:10075E000640119007BAE0FEA3E0FFEFD3946DEED2
:10076E00940640139007BAE0FEA3E0FF90007612C5
:10077E0066E9E599F0800385997480119007BAE0D7
:10078E00FEA3E0FF9000761266E9E599F09007BAB5
:10079E001266D09007BAE0FEA3E0FFEFB40106EEBA
:1007AE00B4070280030209FD900776E0B43C028094
:1007BE00030209FDA22750030208E8C29C900058CC
:1007CE00E0900114F0900059E0900083F090005AF0
:1007DE00E09000A3F090005BE09000CCF090005C05
:1007EE00E0900078F090005DE09000BEF090005E2A
:1007FE00E09000DCF090005FE09000B0F0900060C0
:10080E00E09000CEF0900061E09000FEF09000626B
:10081E00E0900162F0900063E0900163F09000645C
:10082E00E0900164F0123B9D90006AE09000E5F0CC
:10083E0090006BE090009CF090006CE090009DF0BA
:10084E0074639007B6F8E4F0E8A3F074AB9000413F
:10085E00F012044E900041E4F07464F5097508003E
:10086E001200E9A21C4039757301E573D394075049
:10087E002DE5739007B6F8E4F0E8A3F074AA9000A3
:10088E0041F0120115E573C39407500A7464F5091B
:10089E007508001200E97873740126F650CC803783
:1008AE00757308E573D3940E502DE5739007B6F863
:1008BE00E4F0E8A3F074AA900041F0120115E5737C
:1008CE00C3940E500A7464F5097508001200E97895
:1008DE0073740126F650CC0209E7C29C900114E015
:1008EE00900058F0900083E0900059F09000A3E043
:1008FE0090005AF09000CCE090005BF0900078E011
:10090E0090005CF09000BEE090005DF09000DCE0A6
:10091E0090005EF09000B0E090005FF09000CEE0AE
:10092E00900060F09000FEE0900061F07400900086
:10093E0062F07400900063F07400900064F07463D1
:10094E009007B6F8E4F0E8A3F074AB900041F01213
:10095E00044E900041E4F07464F50975080012002D
:10096E00E9757301E573D394075026E5739007B6C6
:10097E00F8E4F0E8A3F074AA900041F012011574A7
:10098E0064F5097508001200E97873740126F650B3
:10099E00D3D29C7599FB743C900776F0757308E57D
:1009AE0073D3940E5026E5739007B6F8E4F0E8A3DF
:1009BE00F074AA900041F01201157464F5097508DF
:1009CE00001200E97873740126F650D374C89007AC
:1009DE00B6F8E4F0E8A3F080FE74C89007B6F8E429
:1009EE00F0E8A3F0D29C754E00754D007599FB0290
:1009FE000C569007BAE0FEA3E0FFEF4E7006859905
:100A0E00317530009007BAE0FEA3E0FF74016F4E1F
:100A1E00701BAC30AD31AA32AB33ED2BFBEC3AFA96
:100A2E008A068B079000761266E9E599F09007BA70
:100A3E001266D09007BAE0FEA3E0FF74026F4E700C
:100A4E0021AC30AD3174566D4C7006E54F64E660E6
:100A5E00028003124090123B9D854F99754E007592
:100A6E004D00020C569007BAE0FEA3E0FF90007610
:100A7E001266E9E599F09007BA1266D09007BAE0CF
:100A8E00FEA3E0FFAC32AD338F028E038C068D07D2
:100A9E00905FDE126691E493F9740193FEEAD39EA1
:100AAE00EB994009854F99754E00754D00020C5615
:100ABE009007BAE0FEA3E0FF9000761266E9E59992
:100ACE00F09007BA1266D09007BAE0FEA3E0FFEFEF
:100ADE00B40006EEB401028003020C56900051E001
:100AEE00D394C7400B900051E0C394C8F550801AC0
:100AFE00900051E0D39463400B900051E0C3946496
:100B0E00F5508006900051E0F550E55075F002A4C6
:100B1E00FFAEF08F73EF9000761266F4EFFCE0FDFF
:100B2E00EC9000791266F4EDFCE0FDEC2DB5500270
:100B3E008003020C470FEF9000761266F4E573FF08
:100B4E00E0FCEF90007A1266F4ECFFE0FCEFC39C41
:100B5E00B550028003020C47E5739000781266F4DC
:100B6E00E573FFE0FCEF90007B1266F4ECFFE0FC17
:100B7E00EF2CB550028003020C47E57390007C12F7
:100B8E0066F4E0C39550900058F0E57390007D1226
:100B9E0066F4E0C39550900059F0E57390007E1214
:100BAE0066F4E0C3955090005AF0740090005BF02C
:100BBE0074FF90005CF0E5739000801266F4E0C361
:100BCE00955090005DF0E5739000811266F4E0C3DD
:100BDE00955090005EF0E5739000821266F4E0C3CB
:100BEE00955090005FF0E57390007F1266F4E0C3BD
:100BFE0095509007B6F8E4F0E8A3F074AB9000417E
:100C0E00F012044E7464F5097508001200E990079D
:100C1E00B61266D012044E7464F5097508001200FF
:100C2E00E99007B61266D012044E7599F97464F500
:100C3E00097508001200E980FE7599FF7464F509C4
:080C4E007508001200E980FEA8
:0F384A0002069002073B020A00020A73020ABE3E
:100C560022E54D903859F8282873020D699007BA95
:100C6600E0FEA3E0FF9000471266E9E0F5999007E1
:100C7600BA1266D09007BAE0FEA3E0FF74116F4E79
:100C86007003754D00020D69856E99020D69900716
:100C9600BAE0FEA3E0FF9000761266E9E0F599EF70
:100CA600B40107EEB40703754D009007BA1266D07B
:070CB600020D699007BBE08D
:0F385900020C60020C63020C8E020C94020CB97C
:100CBD00903A0CF8282873855399020D5E855F993B
:100CCD00020D5E856199020D5E856599020D5E8549
:100CDD006799807D85689980788569998073856A23
:100CED0099806E900016E0F5998066A236B34007A4
:100CFD007599FAC2368041A226B3400575990F80C9
:100D0D00359007C5E0600A9007C5E024DCF59980B1
:100D1D00169007C6E0600A9007C6E024DEF59980BC
:100D2D0006900045E0F599900045E4F09007C5E484
:100D3D00F09007C6E4F0C2268017856B9980128566
:100D4D006699800D856C9980087599FC8003754DA9
:010D5D000095
:103A0C00020CC4020CCA020CD0020CD6020CDC0252
:103A1C000CE1020CE6020CEB020CF0020CF8020DAD
:0D3A2C0047020D4C020D51020D56020D5BBC
:0B0D5E009007BA1266D08003123A39E9
:03386800020D66E8
:100D690022E537255BFFAE5A50010E9000761266D8
:100D7900E9E0F538E537255BFFAE5A50010E0FBFA4
:100D890000010E9000761266E9E0F539853F3BE5F2
:100D990038B539058538378041E539D39538401D4F
:100DA900E539C39538853AF0A4FFAEF0E53B8E04EA
:100DB9008F05FF1266B2ED2538F537801DE538C37A
:100DC9009539853AF0A4FFAEF0E53B8E048F05FF17
:100DD9001266B2EDF4042538F53722E539D3953892
:100DE900401DE539C39538853AF0A4FFAEF0E53BDF
:100DF9008E048F05FF1266B2ED2538F537801DE5A3
:100E090038C39539853AF0A4FFAEF0E53B8E048FDF
:100E190005FF1266B2EDF4042538F5372290007CFF
:100E2900E0B40170E56775F00A84FF7E008F37E54D
:100E39006775F00A84ADF07C008D3A753F0A755AE2
:100E490005755B24E537C394115005120D6A8006B8
:100E59009005ABE0F537E53790006FF0E56775F081
:100E69000A84FF7E008F37E56775F00A84ADF07C50
:100E7900008D3A753F0A755A05755B5AE537C39473
:100E8900115005120D6A80069005E1E0F537E53746
:100E990090000EF02290007CE0B4016AE56775F0DD
:100EA9000A84FF7E008F37E56775F00A84ADF07C10
:100EB900008D3A753F0A755A05755B36E537C39457
:100EC900115005120D6A80069005BDE0F53785378A
:100ED9004BE56775F00A84FF7E008F37E56775F08B
:100EE9000A84ADF07C008D3A753F0A755A05755B29
:100EF90048E537C394115005120D6A80069005CF55
:100F0900E0F53785374C22E55F75F00484FF7E00F4
:100F19008F37E55F75F00484ADF07C008D3A753F3D
:100F290004755A01755B00E537C3943F5005120DEE
:100F39006A80069001B5E0F5378537297528009054
:100F49000044E075F020A4FFAEF09000C7E08E04E5
:100F59008F05FF1266B28D379000AFE0D3955F50D1
:100F6900030210169000D3E0D3955F4010ED900175
:100F7900B61266F4E0F52B752A0002101390009E54
:100F8900E0D3955F4043E5379001B61266F4E0F58A
:100F990038E5379001D61266F4E0F5399000D3E0D0
:100FA900F404255FF53A90009EE0FE9000D3E0F44A
:100FB900042EF53BE538B539058538378003120D20
:100FC900E485372B752A008041E5379001D61266F2
:100FD900F4E0F538E5379001F61266F4E0F539905A
:100FE900009EE0F404255FF53A9000AFE0FE900022
:100FF9009EE0F4042EF53BE538B539058538378090
:1010090003120DE485372B752A000210BD9000D616
:10101900E0D3955F5011E5379002361266F4E0F59A
:101029002B752A000210BD90009FE0D3955F5043B5
:10103900E5379002161266F4E0F538E53790023686
:101049001266F4E0F53990009FE0F404255FF53A63
:101059009000D6E0FE90009FE0F4042EF53BE538C1
:10106900B539058538378003120DE485372B752A84
:10107900008041E5379001F61266F4E0F538E5376E
:101089009002161266F4E0F5399000AFE0F40425F9
:101099005FF53A90009FE0FE9000AFE0F4042EF572
:1010A9003BE538B539058538378003120DE48537B6
:1010B9002B752A00229000E7E0F53C753F11755A1F
:1010C90002755B00AE52AF53E53C75F00FA4FDAC61
:1010D900F0EDD39FEC9E4021E53C8E048F05FF1275
:1010E90066B2ED75F010A4FFAEF0E55F75F01184FE
:1010F900FD7C00ED2FF53D800EE55F75F01184FF55
:101109007E00EF24F0F53D853D37E55F75F01184EC
:10111900AFF07E008F3A120D6A85373EAE52AF535B
:101129009000E7E075F00FA4FDACF0EDD39FEC9EC5
:101139004028755A02755B10853D37120D6A853E48
:1011490038853739AE52AF53E53C8E048F05FF120F
:1011590066DD8D3A853C3B120DE4853729752800FB
:10116900752B64752A00229000E7E0F53C753F1164
:10117900755A02755B00AE52AF53E53C75F00FA48A
:10118900FDACF0EDD39FEC9E4021E53C8E048F052C
:10119900FF1266B2ED75F010A4FFAEF0E56175F0CF
:1011A9001184FD7C00ED2FF53D800EE56175F01190
:1011B90084FF7E00EF24F0F53D853D37E56175F04C
:1011C9001184AFF07E008F3A120D6A85373EAE5218
:1011D900AF539000E7E075F00FA4FDACF0EDD39F9D
:1011E900EC9E4028755A02755B10853D37120D6AD1
:1011F900853E38853739AE52AF53E53C8E048F05AD
:10120900FF1266DD8D3A853C3B120DE48537297561
:101219002800E56B6017E56BC394FE50109000DB66
:10122900E0B402099000C9E0D3940B50028017AED4
:1012390028AF29E56B1266C274E78E048F05FF1289
:1012490066B28C288D299000B1E0B40453E55F752E
:10125900F00484FF7E008F37E55F75F00484ADF0FC
:101269007C008D3A753F04755A01755B00E537C3FB
:10127900943F5005120D6A80069001B5E0F537AE2E
:1012890028AF29E5371266C274648E048F05FF12F0
:1012990066B2AE28AF29EF2DFDEE3CFC8C288D29D6
:1012A900752B64752A002290007CE0B40146E5673D
:1012B90075F00A84FF7E008F37E56775F00A84AD03
:1012C900F07C008D3A753F0A755A05755B00E53764
:1012D900C394115005120D6A8006900587E0F53711
:1012E900AE2AAF2BE5372FFF50010E746412670643
:1012F9008E2A8F2B90007DE0B40146E56875F00ACF
:1013090084FF7E008F37E56875F00A84ADF07C00B4
:101319008D3A753F0A755A05755B6CE537C39411AB
:101329005005120D6A80069005F3E0F537AE2AAF35
:101339002BE5372FFF50010E74641267068E2A8F32
:101349002B90008CE0B40249E56AC3944175F0051D
:1013590084FF7E008F37E56A75F00584ADF07C0067
:101369008D3A753F05755A06755B00E537C39413C9
:101379005005120D6A8006900689E0F537AE2AAF4E
:101389002BE5372FFF50010E74641267068E2A8FE2
:101399002B9000CEE0B40202800302144FE55F7582
:1013A900F01584FF7E008F37E55F75F01584ADF089
:1013B9007C008D3A753F15755A03755BF4E537C3A3
:1013C900940B5005120D6A8006900475E0F537E517
:1013D9003775F0FFA4FFAEF09000CFE08E048F05C3
:1013E900FF1266B2ED900068F0E56675F078A4FF2B
:1013F900AEF074FF8E048F05FF1266B28C5A8D5BB6
:1014090074028C068D071200398F37AC5AAD5B74A4
:1014190004FF1266DD8D3A753F04755A06755B281F
:10142900E537C3941D5005120D6A80069006BBE08E
:10143900F537AE2AAF2BE5372FFF50010E74641232
:1014490067068E2A8F2B90007BE0B4025DE56175FB
:10145900F064A4FFAEF074081200398E5C8F5D74DD
:10146900058E048F05FF1266B28D37AE5CAF5D74D1
:10147900058E048F05FF1266DD8D3A753F05755A95
:1014890005755BDEE537C394135005120D6A8006B6
:10149900900667E0F537AE2AAF2BE5372FFF5001ED
:1014A9000E74641267068E2A8F2B9000BDE0703C83
:1014B900900044E075F00584FF7E008F379000446A
:1014C900E075F00584ADF07C008D3A753F05755ADD
:1014D90005755BC0E537C3941D5005120D6A80067A
:1014E900900653E0F537E537900070F022900084BC
:1014F900E0B401179007C1E0252BFFAE2A50010E79
:101509009000D8E01267068E2A8F2B9000FCE0B479
:1015190001149000FDE0A852B8000495535007E566
:101529005FC39560400280129000A6E0252BFFAEB4
:101539002A50010E8E2A8F2B802F900084E0B4034D
:1015490016A229B3B350109007C4E0C39405A8525A
:10155900B800069553400280109000A6E0252BFFA5
:10156900AE2A50010E8E2A8F2B90007EE0B4020223
:1015790080030218F4900081E0602FE567D3944658
:10158900402890000FE0FEA3E0FF9000BCE075F05A
:1015990003A4FDACF0EFD39DEE9C400E9000E0E07B
:1015A900A852B80005D3955350030218F49000B11E
:1015B900E0B40302800302175885615B755A0090F5
:1015C9000088E0A852B800049553500E900089E0B5
:1015D900A85AB80005D3955B5003021755E5617504
:1015E900F002A4FFAEF074158E048F05FF1266B2E7
:1015F9008C068D079006061266E9FEE0FFEE900064
:1016090080E0FEEF8E0088F0A4FFAEF074648E04D3
:101619008F05FF1266B28C5A8D5B900044E075F01D
:1016290018A4FFAEF09000C7E08E048F05FF126684
:10163900B28C068D0790061E1266E9AE5AAF5BE0C2
:101649001266C274648E048F05FF1266B28C5A8DBD
:101659005BE565A85AB80077D3955B4072E565C329
:10166900955BFFE4955AFE8E5A8F5B7428BE000382
:101679009F500C755B28755A00740D900045F0AEAB
:101689005AAF5B900081E01266C274288E048F0500
:10169900FF1266B28C5A8D5BAE28AF29740A8E048C
:1016A9008F05FF1266B28D068C07AC5AAD5BCFCEA3
:1016B900CF120003740A8E048F05FF1266B28C5A8A
:1016C9008D5BAE28AF2912670E8E288F29807DE5A4
:1016D90065A85AB80004955B5072AE5AAF5BE565D0
:1016E9001267068E5A8F5B7428BE00039F500C75D3
:1016F9005B28755A00740D900045F0AE5AAF5B90A7
:101709000081E01266C274288E048F05FF1266B24A
:101719008C5A8D5BAE28AF29740A8E048F05FF128F
:1017290066B28D068C07AC5AAD5BCFCECF120003E3
:10173900740A8E048F05FF1266B28C5A8D5BAE282F
:10174900AF29EF2DFDEE3CFC8C288D290218F49071
:1017590000C9E0855FF0A4FFAEF074051266C2749B
:10176900071200398E5A8F5B900088E0A852B800A2
:101779000495535012900089E075F002A4FDACF075
:10178900EFC39DEE9C40030218F4E55F75F00B84EE
:10179900FF7E009006061266E9FEE0FFEE900080EB
:1017A900E0FEEF8E0088F0A4FFAEF074648E048F23
:1017B90005FF1266B28C5A8D5B900044E075F018F3
:1017C900A4FFAEF09000C7E08E048F05FF1266B249
:1017D9008C068D0790061E1266E9AE5AAF5BE012C1
:1017E90066C274648E048F05FF1266B28C5A8D5BD3
:1017F900E565A85AB80077D3955B4072E565C3954E
:101809005BFFE4955AFE8E5A8F5B7428BE00039FD6
:10181900500C755B28755A00740D900045F0AE5A4E
:10182900AF5B900081E01266C274288E048F05FFB9
:101839001266B28C5A8D5BAE28AF29740A8E048F5A
:1018490005FF1266B28D068C07AC5AAD5BCFCECFC1
:10185900120003740A8E048F05FF1266B28C5A8D2A
:101869005BAE28AF2912670E8E288F29807DE5652A
:10187900A85AB80004955B5072AE5AAF5BE5651281
:1018890067068E5A8F5B7428BE00039F500C755BE8
:1018990028755A00740D900045F0AE5AAF5B900060
:1018A90081E01266C274288E048F05FF1266B28C1D
:1018B9005A8D5BAE28AF29740A8E048F05FF126614
:1018C900B28D068C07AC5AAD5BCFCECF1200037434
:1018D9000A8E048F05FF1266B28C5A8D5BAE28AF53
:1018E90029EF2DFDEE3CFC8C288D29229000DCE0AF
:1018F900B4026AE55F75F00884FF7E008F37E55F03
:1019090075F00884ADF07C008D3A753F08755A0171
:10191900755BE0E537C3943F5005120D6A80069068
:101929000275E0F53785372D752C00AE2CAF2DAC3F
:101939002AAD2B12000374648E048F05FF1266B260
:101949008C2C8D2D900079E08C068D071266C2745F
:10195900648E048F05FF1266B28C2C8D2DAE28AFD4
:1019690029AC2AAD2B12000374648E048F05FF1273
:1019790066B28C288D29900079E08C068D07126655
:10198900C274648E048F05FF1266B28C288D29A259
:101999000D401DAE52AF537405BE00039F5002D2D5
:1019A9000DE561D394CC4008D2017411900045F043
:1019B9009000DBE0B402089000C9E0640B6002808B
:1019C90035AE28AF29E56B1266C274E78E048F0520
:1019D900FF1266B28C288D299000DCE0B40217AEA4
:1019E9002CAF2DE56B1266C274E78E048F05FF12CA
:1019F90066B28C2C8D2D90009BE05402601B9000E8
:101A090092E0A852B80012D39553400DA20DB3B37A
:101A19005007E561C3949A40028028AE34AF3590EF
:101A29000090E075F002A4FDACF0EF2DFDEE3CFC5A
:101A390074022DFD50010CE561BC0007D39D4003E4
:101A4900754301856135753400E5437003021B3820
:101A59009000EEE0C395435003021B2A9000FEE07C
:101A6900C394025076E56775F00A84FF7E009005FD
:101A7900761266E9E0F55B755A00AE5AAF5B9000E5
:101A890091E01266C274648E048F05FF1266B28CEF
:101A99005C8D5D9000EEE004C395438C068D0712C2
:101AA90066C29000EEE08E048F05FF1266B28C5C70
:101AB9008D5DAE28AF29EF2DFDEE3CFC8C288D29DC
:101AC9009000DCE0B40212AE2CAF2DAA5CAB5DEF46
:101AD9002BFBEE3AFA8A2C8B2D80469000EEE0041F
:101AE900C39543854BF0A4FFAEF09000EEE08E0461
:101AF9008F05FF1266B28C5C8D5DAE28AF29EF2D84
:101B0900FDEE3CFC8C288D299000DCE0B40212AE7D
:101B19002CAF2DAA5CAB5DEF2BFBEE3AFA8A2C8B2E
:101B29002D05439000EEE0C39543500375430090A3
:101B3900009BE05401601B90008FE0A852B800128E
:101B4900D39553400DA20DB3B35007E55FC394CCB1
:101B59004002802590008DE075F003A4FFAEF0E50A
:101B6900402FFF50010E74032FFF50010EE55FBE99
:101B79000007D39F4003754401855F40E544700326
:101B8900021C6B9000EFE0C395445003021C5D906A
:101B990000FEE0C394025076E56775F00A84FF7E83
:101BA900009005761266E9E0F55B755A00AE5AAF0A
:101BB9005B90008EE01266C274648E048F05FF127A
:101BC90066B28C5C8D5D9000EFE004C395448C0691
:101BD9008D071266C29000EFE08E048F05FF126632
:101BE900B28C5C8D5DAE28AF29EF2DFDEE3CFC8CEF
:101BF900288D299000DCE0B40212AE2CAF2DAA5C2E
:101C0900AB5DEF2BFBEE3AFA8A2C8B2D80469000C8
:101C1900EFE004C39544854CF0A4FFAEF09000EFCB
:101C2900E08E048F05FF1266B28C5C8D5DAE28AF25
:101C390029EF2DFDEE3CFC8C288D299000DCE0B4C9
:101C49000212AE2CAF2DAA5CAB5DEF2BFBEE3AFA7C
:101C59008A2C8B2D05449000EFE0C3954450037501
:101C690044009000F1E02529FFAE2850010E8E288E
:101C79008F299000A0E0A828B80004952950099060
:101C890000A0E0F5297528009000DCE0B4020D9071
:101C990000A0E0A82CB80006952D4002800990000C
:101CA900A0E0F52D752C00229000DCE0B401028043
:101CB90003021DBCA20DB35003021DBA9000A7E098
:101CC900B40168AE28AF29AC52AD53120003743C7D
:101CD9008E048F05FF1266B29000B7E0BC00109D1C
:101CE900400D9000B9E0A828B8000495295002D207
:101CF90002AE28AF29AC52AD53120003743C8E04D6
:101D09008F05FF1266B29000B7E0C3940ABC0015B4
:101D1900D39D40119000B9E0C39405A828B80005E7
:101D2900D3952950028002C2028068AE28AF29AC3F
:101D390052AD5312000374788E048F05FF1266B2F8
:101D49009000B7E0BC00109D400D9000B9E0A828B4
:101D5900B8000495295004D2028038AE28AF29ACC6
:101D690052AD5312000374788E048F05FF1266B2C8
:101D79009000B7E0C3940ABC0015D39D40119000B0
:101D8900B9E0C39405A828B80005D3952950028065
:101D990002C202A202B34019AE28AF299000B8E0EE
:101DA9001266C274648E048F05FF1266B28C288D88
:101DB900298002C202A200B34006A201B3B35009AE
:101DC900900015E4F0A3F08024AE28AF297400D365
:101DD9009F74019E400C900015E528F0A3E529F0B9
:101DE900800B74FF900015F8E4F0E8A3F09000BEB2
:101DF900E0D39402400C9000A9E07006A20DB3B3A1
:101E09004002801AAE28AF2974021266C28E288F4A
:101E190029AE2CAF2D74021266C28E2C8F2D900024
:101E2900A7E0B4011AAE28AF2974021266C28E283F
:101E39008F29AE2CAF2D74021266C28E2C8F2DAE57
:101E490028AF29745E1266C2740A8E048F05FF12C8
:101E590066B28C288D299000DCE0B40217AE2CAF55
:101E69002D745E1266C2740A8E048F05FF1266B263
:101E79008C2C8D2DAE28AF297402BE000AD39F4049
:101E890006752902752800AE2CAF2D7402BE000A12
:101E9900D39F4006752D02752C00900013E528F09C
:101EA900A3E529F022900044E09003761266F4E05D
:101EB900F541754264900044E0FE9000B2E0D39E83
:101EC9004037E55F75F00884FF7E008F37E55F7561
:101ED900F00884ADF07C008D3A753F08755A03759A
:101EE9005B96E537C3941F5005120D6A800690046E
:101EF9002BE0F5378537428035E55F75F00884FFBB
:101F09007E008F37E55F75F00884ADF07C008D3A6F
:101F1900753F08755A03755BB6E537C3941F5005BD
:101F2900120D6A800690044BE0F5378537422290FE
:101F390000E8E0F53C753F11755A04755B00AE5237
:101F4900AF53E53C75F00FA4FDACF0EDD39FEC9ECB
:101F59004021E53C8E048F05FF1266B2ED75F01045
:101F6900A4FFAEF0E55F75F01184FD7C00ED2FF55F
:101F79003D800EE55F75F01184FF7E00EF24F0F5DA
:101F89003D853D37E55F75F01184AFF07E008F3AEE
:101F9900120D6A85373EAE52AF539000E8E075F0F6
:101FA9000FA4FDACF0EDD39FEC9E4028755A047543
:101FB9005B10853D37120D6A853E38853739AE523B
:101FC900AF53E53C8E048F05FF1266DD8D3A853CE3
:101FD9003B120DE4853741754264229000E8E0F533
:101FE9003C753F11755A04755B00AE52AF53E53C21
:101FF90075F00FA4FDACF0EDD39FEC9E4021E53CBC
:102009008E048F05FF1266B2ED75F010A4FFAEF0D5
:10201900E56175F01184FD7C00ED2FF53D800EE53D
:102029006175F01184FF7E00EF24F0F53D853D37A1
:10203900E56175F01184AFF07E008F3A120D6A8563
:10204900373EAE52AF539000E8E075F00FA4FDACF7
:10205900F0EDD39FEC9E4028755A04755B10853DC1
:1020690037120D6A853E38853739AE52AF53E53C94
:102079008E048F05FF1266DD8D3A853C3B120DE417
:102089008537417542649000B1E0B4047990004409
:10209900E0FE9000B2E0D39E4037E55F75F008841A
:1020A900FF7E008F37E55F75F00884ADF07C008D09
:1020B9003A753F08755A03755B96E537C3941F5007
:1020C90005120D6A800690042BE0F53785374280AA
:1020D90035E55F75F00884FF7E008F37E55F75F0A1
:1020E9000884ADF07C008D3A753F08755A03755B1D
:1020F900B6E537C3941F5005120D6A800690044B4C
:10210900E0F5378537422290007CE0B4013BE56772
:1021190075F00A84FF7E008F37E56775F00A84AD94
:10212900F07C008D3A753F0A755A05755B12E537E3
:10213900C394115005120D6A8006900599E0F53790
:10214900E5422537C39464F54290007DE0B4013B34
:10215900E56875F00A84FF7E008F37E56875F00A37
:1021690084ADF07C008D3A753F0A755A05755B7E22
:10217900E537C394115005120D6A8006900605E0F3
:10218900F537E5422537C39464F542E5412542F523
:1021990036900084E0B402109007C0E02536FE9026
:1021A90000D8E0F4042EF5369000DBE0D39401402A
:1021B90040E56BC394E7501D74E7C3956BFE900728
:1021C900C2E08E00F5F0E884FF7E008F37E5362502
:1021D90037F536801CE56BC394E7FE9007C2E08EA5
:1021E90000F5F0E884FF7E008F37E536C39537F5B3
:1021F90036A20D4006E5412464F536E536D39464EC
:102209004009E536C39464F53680037536009000BD
:10221900B4E0C3953650069000B4E0F53622D200FA
:1022290090006EE0A852B800049553504190006E9A
:10223900E0A852B800049553500375360F90006E0C
:10224900E004A852B800049553500375360A90006B
:102259006EE02402A852B80004955350057536055E
:10226900C20090006EE060067409900045F0C23922
:102279007E017F009000BAE01266C29000C9E08E2C
:10228900048F05FF1266B2E55FBC0017D39D4013AA
:102299009000C3E0B40204D2398002C200740A90EB
:1022A9000045F09000BBE0C3956750159000CDE064
:1022B900A852B8000495535002C200740B9000450F
:1022C900F0E567C39464501D900113E0600D90011F
:1022D90013E0A852B80006955340028008C2007462
:1022E9000B900045F0A20040037536059000FCE014
:1022F900B401149000FDE0A852B8000495535007AA
:10230900E55FC39560400280089000A5E0F536803E
:102319003A900084E0B40306A229B3B34002802BAB
:102329009007C4E0C39405A852B800049553500C13
:102339009000A5E0F536740C900045F09007C4E0D4
:10234900A852B8000495535002C20085366C90001B
:1023590076E02536FE900044E075F01E84FC7F008F
:10236900EE2CF53622900044E075F00584FF7E00DE
:102379008F37900044E075F00584ADF07C008D3A0C
:10238900753F05755A03755BD69000C7E01475F063
:102399000584FF7E00E537BE00039F5005120D6AD4
:1023A900800BE53790044C1266F4E0F537E5379079
:1023B90007C3F09007C3E0FE9000B6E0C39E500843
:1023C9009000B6E09007C3F022E56775F00A84FF34
:1023D9007E009005761266E9E0F546E546D39464F9
:1023E9004010E546C3946475F00F84FF7E008F4664
:1023F9008003754600900099E02546F54622900035
:10240900B1E0C3940350269007B0E0FEA3E0FF7447
:1024190004120039E55F1266C2740F8E048F05FF3E
:102429001266B29007AEECF0A3EDF080249007B0ED
:10243900E0FEA3E0FF7404120039E5611266C2747C
:102449000F8E048F05FF1266B29007AEECF0A3ED74
:10245900F090008CE0B40262E56AC3944175F0051E
:1024690084FF7E008F37E56A75F00584ADF07C0046
:102479008D3A753F05755A06755B14E537C3941790
:102489005005120D6A800690069DE0F5379007AE5B
:10249900E0FEA3E0FF740A8E048F05FF1266B2E521
:1024A900378C068D071266C2740A8E048F05FF12D7
:1024B90066B29007AEECF0A3EDF09007AEE0FEA394
:1024C900E0FF9007B4E0FCA3E0FDEDD39FEC9E4054
:1024D9000F9007B4E0F8A3E09007AEC8F0A3C8F0E6
:1024E900229006BDE090386BF8282873804C8553FC
:1024F9007380479000C9E0855FF0A4FFAEF07408CF
:102509001200398F738033856173802E85677380DC
:10251900298568738024856973801F856A73801A89
:10252900856B7380158566738010856573800B854F
:0A2539006C738006900016E0F57345
:10386B000224F50224F70224FC022510022515027E
:10387B00251A02251F02252402252902252E0225A1
:07388B003302253802253D40
:102543009006BEE0FE9006BFE0D39E404B9006BDD2
:10255300E0B404189006BFE0C395735002D22A90EA
:1025630006BEE0D395734002C22A802A9006BEE0DD
:10257300C3957350099006BFE0D395735002800250
:10258300D22A9006BEE0D3957350099006BFE0C3EC
:1025930095735002C22A802A9006BEE0D3957340F9
:1025A300099006BFE0C3957340028002C22A9006D9
:1025B300BEE0C3957340099006BFE0D39573400214
:1025C300D22A229006C1E0903892F8282873804CD2
:1025D30085537380479000C9E0855FF0A4FFAEF098
:1025E30074081200398F738033856173802E856779
:1025F3007380298568738024856973801F856A7356
:10260300801A856B7380158566738010856573806A
:0C2613000B856C738006900016E0F573D8
:103892000225D10225D30225D80225EC0225F10208
:1038A20025F60225FB02260002260502260A02262A
:0738B2000F02261402261983
:10261F009006C2E0FE9006C3E0D39E405F9006C1D5
:10262F00E0B404189006C3E0C395735002D22B9008
:10263F0006C2E0D395734002C22B803E9006C2E0E3
:10264F00C3957350099006C3E0D39573500280026F
:10265F00D22B9006C2E0D3957350099006C3E0C306
:10266F0095735002C22B9006C1E0B401099000D5BA
:10267F00E0D3956150028002C22B802A9006C2E0FF
:10268F00D3957340099006C3E0C39573400280024F
:10269F00C22B9006C2E0C3957340099006C3E0D3E6
:1026AF0095734002D22B229006C5E09038B9F828D6
:1026BF002873804C85537380479000C9E0855FF085
:1026CF00A4FFAEF074081200398F738033856173E5
:1026DF00802E856773802985687380248569738050
:1026EF001F856A73801A856B7380158566738010DA
:1026FF00856573800B856C738006900016E0F5730B
:1038B9000226C10226C30226C80226DC0226E1022C
:1038C90026E60226EB0226F00226F50226FA022651
:0738D900FF0227040227098A
:10270F009006C6E0FE9006C7E0D39E404B9006C5EC
:10271F00E0B404189006C7E0C395735002D22C9012
:10272F0006C6E0D395734002C22C802A9006C6E0FD
:10273F00C3957350099006C7E0D39573500280027A
:10274F00D22C9006C6E0D3957350099006C7E0C30C
:10275F0095735002C22C802A9006C6E0D395734021
:10276F00099006C7E0C3957340028002C22C900601
:10277F00C6E0C3957340099006C7E0D39573400236
:10278F00D22C229006C9E09038E0F8282873804CAC
:10279F0085537380479000C9E0855FF0A4FFAEF0CA
:1027AF0074081200398F738033856173802E8567AB
:1027BF007380298568738024856973801F856A7388
:1027CF00801A856B7380158566738010856573809D
:0C27DF000B856C738006900016E0F5730B
:1038E00002279D02279F0227A40227B80227BD02B4
:1038F00027C20227C70227CC0227D10227D60227D8
:07390000DB0227E00227E5CE
:1027EB009006CAE0FE9006CBE0D39E404B9006C904
:1027FB00E0B404189006CBE0C395735002D22D9031
:10280B0006CAE0D395734002C22D802A9006CAE017
:10281B00C3957350099006CBE0D395735002800299
:10282B00D22D9006CAE0D3957350099006CBE0C326
:10283B0095735002C22D802A9006CAE0D39573403F
:10284B00099006CBE0C3957340028002C22D90061F
:10285B00CAE0C3957340099006CBE0D39573400251
:10286B00D22D229006CDE0903907F8282873804CA2
:10287B0085537380479000C9E0855FF0A4FFAEF0ED
:10288B0074081200398F738033856173802E8567CE
:10289B007380298568738024856973801F856A73AB
:1028AB00801A856B738015856673801085657380C0
:0C28BB000B856C738006900016E0F5732E
:1039070002287902287B022880022894022899023B
:10391700289E0228A30228A80228AD0228B202285E
:07392700B70228BC0228C111
:1028C7009006CEE0FE9006CFE0D39E404B9006CD1B
:1028D700E0B404189006CFE0C395735002D22E904F
:1028E70006CEE0D395734002C22E802A9006CEE032
:1028F700C3957350099006CFE0D3957350028002B9
:10290700D22E9006CEE0D3957350099006CFE0C340
:1029170095735002C22E802A9006CEE0D39573405D
:10292700099006CFE0C3957340028002C22E90063D
:10293700CEE0C3957340099006CFE0D3957340026C
:10294700D22E229006D1E090392EF8282873804C99
:1029570085537380479000C9E0855FF0A4FFAEF010
:1029670074081200398F738033856173802E8567F1
:102977007380298568738024856973801F856A73CE
:10298700801A856B738015856673801085657380E3
:0C2997000B856C738006900016E0F57351
:10392E0002295502295702295C02297002297502C3
:10393E00297A02297F02298402298902298E0229E5
:07394E009302299802299D54
:1029A3009006D2E0FE9006D3E0D39E404B9006D132
:1029B300E0B404189006D3E0C395735002D22F906D
:1029C30006D2E0D395734002C22F802A9006D2E04C
:1029D300C3957350099006D3E0D3957350028002D8
:1029E300D22F9006D2E0D3957350099006D3E0C35B
:1029F30095735002C22F802A9006D2E0D39573407C
:102A0300099006D3E0C3957340028002C22F90065B
:102A1300D2E0C3957340099006D3E0D39573400287
:102A2300D22F229006D5E0903955F8282873804C90
:102A330085537380479000C9E0855FF0A4FFAEF033
:102A430074081200398F738033856173802E856714
:102A53007380298568738024856973801F856A73F1
:102A6300801A856B73801585667380108565738006
:0C2A73000B856C738006900016E0F57374
:10395500022A31022A33022A38022A4C022A51024B
:103965002A56022A5B022A60022A65022A6A022A6C
:073975006F022A74022A7997
:102A7F009006D6E0FE9006D7E0D39E404B9006D549
:102A8F00E0B404189006D7E0C395735002D230908B
:102A9F0006D6E0D395734002C230802A9006D6E066
:102AAF00C3957350099006D7E0D3957350028002F7
:102ABF00D2309006D6E0D3957350099006D7E0C375
:102ACF0095735002C230802A9006D6E0D39573409A
:102ADF00099006D7E0C3957340028002C23090067A
:102AEF00D6E0C3957340099006D7E0D395734002A3
:102AFF00D230229006D9E090397CF8282873804C88
:102B0F0085537380479000C9E0855FF0A4FFAEF056
:102B1F0074081200398F738033856173802E856737
:102B2F007380298568738024856973801F856A7314
:102B3F00801A856B73801585667380108565738029
:0C2B4F000B856C738006900016E0F57397
:10397C00022B0D022B0F022B14022B28022B2D02D3
:10398C002B32022B37022B3C022B41022B46022BF3
:07399C004B022B50022B55DA
:102B5B009006DAE0FE9006DBE0D39E404B9006D960
:102B6B00E0B404189006DBE0C395735002D23190A9
:102B7B0006DAE0D395734002C231802A9006DAE080
:102B8B00C3957350099006DBE0D395735002800216
:102B9B00D2319006DAE0D3957350099006DBE0C38F
:102BAB0095735002C231802A9006DAE0D3957340B8
:102BBB00099006DBE0C3957340028002C231900698
:102BCB00DAE0C3957340099006DBE0D395734002BE
:102BDB00D231229006DDE09039A3F8282873804C7F
:102BEB0085537380479000C9E0855FF0A4FFAEF07A
:102BFB0074081200398F738033856173802E85675B
:102C0B007380298568738024856973801F856A7337
:102C1B00801A856B7380158566738010856573804C
:0C2C2B000B856C738006900016E0F573BA
:1039A300022BE9022BEB022BF0022C04022C09025E
:1039B3002C0E022C13022C18022C1D022C22022C7A
:0739C30027022C2C022C311D
:102C37009006DEE0FE9006DFE0D39E404B9006DD77
:102C4700E0B404189006DFE0C395735002D23290C7
:102C570006DEE0D395734002C232802A9006DEE09A
:102C6700C3957350099006DFE0D395735002800235
:102C7700D2329006DEE0D3957350099006DFE0C3A9
:102C870095735002C232802A9006DEE0D3957340D6
:102C9700099006DFE0C3957340028002C2329006B6
:102CA700DEE0C3957340099006DFE0D395734002D9
:102CB700D232229006E1E09039CAF8282873804C76
:102CC70085537380479000C9E0855FF0A4FFAEF09D
:102CD70074081200398F738033856173802E85677E
:102CE7007380298568738024856973801F856A735B
:102CF700801A856B73801585667380108565738070
:0C2D07000B856C738006900016E0F573DD
:1039CA00022CC5022CC7022CCC022CE0022CE502E8
:1039DA002CEA022CEF022CF4022CF9022CFE022D06
:0739EA0003022D08022D0D60
:102D13009006E2E0FE9006E3E0D39E404B9006E18E
:102D2300E0B404189006E3E0C395735002D23390E5
:102D330006E2E0D395734002C233802A9006E2E0B4
:102D4300C3957350099006E3E0D395735002800254
:102D5300D2339006E2E0D3957350099006E3E0C3C3
:102D630095735002C233802A9006E2E0D3957340F4
:102D7300099006E3E0C3957340028002C2339006D4
:102D8300E2E0C3957340099006E3E0D395734002F4
:102D9300D23322AE2EAF2F74F5D39F74019E400819
:102DA300782E126716022EB0752F01752E00AE52C3
:102DB300AF53E546BE000DD39F40099000ABE0D36F
:102DC300954740028023754700E546C39553F57345
:102DD3009000AEE0D395454008E5452573F5458061
:102DE300069000AEE0F54580020547900087E0D3EA
:102DF3009561401CE55FC395604015AE52AF53E546
:102E030046BE00039F50099000ACE0D395484002B2
:102E1300806E9007C7E0A852B8000495535003751D
:102E23004A009007C7E0A852B8000BD39553400659
:102E3300E5539007C7F0E54A7041E553C39546F55E
:102E430073E573D3940540037573059000ADE0C338
:102E530095455007E573C3954540028009E545C391
:102E63009573F54580069000ADE0F5459000ADE023
:102E7300D3954540069000ADE0F5457548008002C6
:102E83000548E54A7016900087E0C39561500DE54B
:102E9300462405A852B8000695534002800F9000BF
:102EA3009AE0F545754A0174789007C7F022AE2E73
:102EB300AF2F74E9D39F74039E4008782E126716D0
:102EC30002304F752F01752E00754532A234402A0A
:102ED30075451990009AE075F002A4FFAEF0E5473E
:102EE300BE0006D39F4002D2340547754A03747867
:102EF3009007C7F075490002303EAE52AF53E54626
:102F03006F4E700302303EE546BE000DD39F40096D
:102F13009000ABE0D395474002800F754700E54A28
:102F2300C394035003754519800DE546C39553F5C6
:102F330073E5472573F547900087E0D39561400E0D
:102F43009007C7E0A852B80007D395534002800CFE
:102F5300054990009AE0B54903754A00E54AB40370
:102F630006A20DB3B34002800A0549E549B43C0308
:102F7300754A02E54AB402299007C7E0A852B8008F
:102F83000ED395534009E5539007C7F07549009058
:102F93000087E0C39561500975490074789007C7AD
:102FA300F0E54A705A900087E0D39561401CE55FD5
:102FB300C395604015AE52AF53E546BE00039F5024
:102FC300099000ACE0D3954840028008754800752D
:102FD300454B8028E553C39546F573E573D39405B4
:102FE3004003757305900087E0D395614008E54879
:102FF3002573F5488006E5482406F548754900E53C
:103003004A7016900087E0C39561500DE54624058C
:10301300A852B80006955340028003754A01E54A59
:10302300B40118754519054990009AE0B54906752C
:103033004A0275490074789007C7F0E54575F00AB0
:10304300A4FFAEF09007B8EEF0A3EFF022E56F9087
:1030530039F1F828287390007FE0700302327790EB
:1030630000B5E0B401028003023192900042E0B562
:103073005E02800302318F7E017F00E5BE1266C2CD
:10308300E5BD2FFF50010E8E5A8F5B74101266C27E
:1030930090006DE08E048F05FF1266B29007BCECC2
:1030A300F0A3EDF074FFBC00039D500B74FF900779
:1030B300BCF8E4F0E8A3F0E56B600FE56BC394FEA6
:1030C30050089000DBE06402600280649000C9E075
:1030D300B40B1F9007BCE0FEA3E0FF74E71266C2C7
:1030E300E56B8E048F05FF1266B29007BCECF0A36C
:1030F300EDF09000C9E0D3940B40089000B1E06478
:10310300046002802B9007BCE0FEA3E0FF9007BEA3
:10311300E0FCA3E0FDEFD39DEE9C400D12670E9003
:1031230007BCEEF0A3EFF080079007BCE4F0A3F038
:1031330090007FE0B4021E9007BCE0FEA3E0FF9086
:1031430007C8E02FFF50010E74011200399007BC2D
:10315300EEF0A3EFF09007BCE0FEA3E0FF9007C8FA
:10316300E0BE0008D39F4004D2378002B2379007F5
:10317300BDE09007C8F09000B1E064016006A2379B
:10318300B3B3400280069007BDE0F55F023275D20B
:10319300377E017F00E5BE1266C2E5BD2FFF5001F9
:1031A3000E8E5A8F5B74101266C290006DE08E040F
:1031B3008F05FF1266B29007BCECF0A3EDF0E56B50
:1031C300600FE56BC394FE50089000DBE06402607F
:1031D3000280649000C9E0B40B1F9007BCE0FEA31B
:1031E300E0FF74E71266C2E56B8E048F05FF12667B
:1031F300B29007BCECF0A3EDF09000C9E0D3940BC0
:1032030040089000B1E064046002802B9007BCE0AA
:10321300FEA3E0FF9007BEE0FCA3E0FDEFD39DEE2D
:103223009C400D12670E9007BCEEF0A3EFF08007F1
:103233009007BCE4F0A3F090007FE0B4021E900777
:10324300BCE0FEA3E0FF9007C8E02FFF50010E741F
:10325300011200399007BCEEF0A3EFF09007BDE038
:103263009007C8F09000B1E0640160069007BDE0EC
:10327300F55F8003755F0090007BE07006756F015A
:1032830002305075BB1802384590007BE070030292
:1032930033FD7E017F00E5BE1266C2E5BD2FFF5000
:1032A300010E8E5A8F5B9000C1E0B4010F7E0F7F39
:1032B300FFAC5AAD5B12670E8E5A8F5B9000E6E04F
:1032C300B40245AE5AAF5B90001FE0FCA3E0FDEDF6
:1032D300D39FEC9E400A90001FE55AF0A3E55BF0F4
:1032E300AE5AAF5B900021E0FCA3E0FDEFD39DEE6F
:1032F3009C400A900021E55AF0A3E55BF0AE5AAF7B
:103303005B74041200398F619000E6E0704CAE5A92
:10331300AF5B90001FE0FCA3E0FDEFD39DEE9C406C
:103323000912670E8E5A8F5B8006755B00755A0013
:10333300AE5AAF5B74101266C290006AE08E048FBF
:1033430005FF1266B28C5A8D5B74FFBC0009D39DD6
:103353004005855B6180037561FE9000B1E0B401B7
:103363000280030233FBA20DB3B3500E900085E03D
:10337300A852B80005D39553500280719000C2E063
:103383008561F0A4FFAEF074648E048F05FF1266AE
:10339300B28C5A8D5BE56B6016E56BC394FE500FE0
:1033A3009000DBE0B402089000C9E0640B60028087
:1033B30017AE5AAF5B74E71266C2E56B8E048F05D6
:1033C300FF1266B28C5A8D5BAE5AAF5B9007BCE0BE
:1033D300FCA3E0FDEDD39FEC9E4005855B5F800B76
:1033E300A237B340069007BDE0F55F800BA237B369
:1033F30040069007BDE0F55F800375610090007E95
:10340300E07006756F0202305075BB1902384590A3
:10341300007EE070030234B2E55ED39551400302AF
:1034230034B090001DE0FEA3E0FFE565126706904F
:10343300001DEEF0A3EFF07E017F00E5BE1266C231
:10344300E5BD2FFF50010E8E5A8F5B9000EBE070AD
:1034530013740A1266C274518E048F05FF1266B28A
:103463008D658019AE5AAF5B740A1266C28F048EE3
:10347300057E017F95CDCCCD1265B08F65E565D313
:103483009464400375656490001DE0FEA3E0FFE5CE
:10349300652FFF50010E90001DEEF0A3EFF090009A
:1034A30082E0048E048F05FF1266B28D658003757A
:1034B30065329000CEE07006756F0302305075BB25
:1034C300130238459000CEE0604A7E017F00E5BEDE
:1034D3001266C2E5BD2FFF50010E8E5A8F5B740436
:1034E3001200398F669000D0E08566F0A4FDACF041
:1034F3007464FF1266B28D669000CFE08566F0A417
:10350300FFAEF074FF8E048F05FF1266B2ED9000DC
:1035130069F0800375660090007CE07006756F04A7
:1035230002305075BB1702384590007CE0B40102AD
:1035330080030235C07E017F00E5BE1266C2E5BD91
:103543002FFF50010E8E5A8F5B9007C9E0601990D0
:1035530007C9E01490602212008CE493FC74019379
:10356300FDEDC39FEC9E400280069007C9E014F076
:103573009007C9E0C394B3501DAE5AAF5B9007C91F
:10358300E00490602212008CE493FC740193FDEF3D
:10359300C39DEE9C400280069007C9E004F09007AB
:1035A300C9E0FE9000A2E08E0088F0A4FFAEF074A4
:1035B300648E048F05FF1266B28D67800375670002
:1035C30090007DE07006756F0502305075BB1602E2
:1035D300384590007DE0B4010280030236697E0124
:1035E3007F00E5BE1266C2E5BD2FFF50010E8E5A65
:1035F3008F5B9007CAE060199007CAE01490618C52
:1036030012008CE493FC740193FDEDC39FEC9E4088
:103613000280069007CAE014F09007CAE0C394B38F
:10362300501DAE5AAF5B9007CAE00490618C120044
:103633008CE493FC740193FDEFC39DEE9C400280E8
:10364300069007CAE004F09007CAE0FE9000A8E0E5
:103653008E0088F0A4FFAEF074648E048F05FF1211
:1036630066B28D68800375680075BB1F0238457E9E
:10367300017F00E5BE1266C2E5BD2FFF50010E8E2D
:103683005A8F5B74091266C274E68E048F05FF12AB
:1036930066B28D6A900084E07006756F0702305041
:1036A30075BB15023845900084E070030237C47E71
:1036B300017F00E5BE1266C2E5BD2FFF50010E8EED
:1036C3005A8F5B74041200398F69900084E0B4014F
:1036D300159000D8E08569F0A4FFAEF074071200DE
:1036E30039EF9007C1F0900084E0B402159000D840
:1036F300E08569F0A4FFAEF07407120039EF90077C
:10370300C0F0900084E0B4030280030237A7900066
:10371300C5E0701CE569C394195002D229E569D349
:1037230094644002C2299000A4E09007C4F080632F
:103733009000A4E070349000D8E08569F0A4FFAE57
:10374300F074FF8E048F05FF1266B2ED9007C4F08C
:10375300AE52AF53741EBE0006D39F4002D229E57A
:1037630061D394E54002C2298029E569C3940A50D4
:103773000DAE52AF53741EBE0004D39F500280029D
:10378300D229E561D394E54002C2299000A4E090D8
:1037930007C4F09007C4E0C394055006740590076E
:1037A300C4F0C238900084E0B40414E569C39419EA
:1037B3005002D238E569D394324002C238C229801C
:1037C300037569009000DBE07006756F08023050E6
:1037D30075BB14806D9000DBE060567E017F00E5D1
:1037E300BE1266C2E5BD2FFF50010E8E5A8F5BEFEE
:1037F300D39421EE940E4005756BFF8015AE5AAF3E
:103803005B74101266C274E38E048F05FF1266B2F6
:103813008D6BE56B75F00BA4FFAEF09000C9E08EE5
:10382300048F05FF1266B29007BEECF0A3EDF080A3
:1038330003756B0090007FE0600575BB1A8003750C
:02384300BB18B0
:1039F10002305902328C0234120234C702352C02D1
:0B3A010035D50236720236A90237D814
:05384500056FD2EC222A
:0966F4002582F582500205832283
:0F008C0025E050020583258250020583F582226C
:10669100EF2F500205832582F582E5833E2EF58397
:0166A10022D6
:10670600CFC39FFF50011E22C3EF9DFFEE9CFE22CA
:086716000806B6000218062275
:0D66D000A3E004F07006120049E004F0227F
:0E003900048007C3CE13CECF13CFD5E0F6223E
:1065B000BC000FBE0008ED8FF084FFADF022E4FEBA
:1065C000FF22BE000DEF60FE54F0606F20E7030273
:1065D0006666EAC0E0EBC0E078017A0075F001EE93
:1065E00020E710EF25E0FFEE33FE0AC5F023C5F0EB
:1065F00030E7F0EA5407F9096A7A007B0060010885
:10660000C3EC9E40167004ED9F4010ED9FFDEC9E84
:10661000FCE5F0CA4ACA03F5F08005E5F003F5F0A1
:10662000C3EE13FEEF13FFD9D77908CACBCAD8D06F
:10663000EAFEEBFFD0E0FBD0E0FA22EC8FF084FC26
:10664000ED54F045F0C48FF084FEEDC454F045F0F5
:10665000C48FF084FDEEC4FE54F02DFFEE540F3CC9
:10666000FEADF07C0022790078008FF0EC7E0820EF
:10667000E70DC3CD33CD33C933C9C833C8DEF08489
:1066800049F9E5F08FF0BE00E6FD7C00E9FFE8FE89
:0166900022E7
:0E66C200F88FF0A4FFE5F0CE88F0A42EFE22A3
:10000300EF8DF0A4F9A8F0EF8CF0A428F8EE8DF0B2
:06001300A428FEE9FF2213
:1066A200600D782B0266AC007830D8FED5E0F82277
:1066B200EEC0E07E001265B0EFFDEEFCD0E0FE22FF
:0C66DD00EEC0E07E001265B0D0E0FE22AE
:03001B0002001EC2
:0300530002005652
:03009B00020071EF
:030000000266FD98
:0966FD0075817575D00002432C73
:0B66E900E5822FF582E5833EF5832259
:0A0049000582D5820215831582227C
:10001E00C0E0C0F0C083C082C0D075D0001242666E
:0B002E00D0D0D082D083D0F0D0E032E0
:10005600C0E0C0F0C083C082C0D075D00012426933
:10006600D0D0D082D083D0F0D0E032C0E0C0F0C093
:1000760083C082C0D075D0001242EED0D0D082D0DC
:0600860083D0F0D0E0324F
:00000001FF
